:020000041100E9
:1030000070B5402501F0E2F80621002001F06CF9CE
:10301000032007F08DFF154C0223FE212800144ADF
:10302000257401F033F900281DD10223FF21114A34
:10303000207C01F02BF9002815D10F4B0F4A1B689B
:10304000934205D9C02204212800920001F06CF9B6
:103050002368002B04D10C222000094908F028F92C
:1030600001F002F970BD00232374F9E7F462FF1F39
:103070000063FF1F0263FF1F2463FF1F871300000D
:1030800038B50011F7B5164B0192C318021D002088
:10309000009388235B05D3181B685C1C1AD09CB274
:1030A000402C18D88D781E0CAC466746CD782D0282
:1030B0003D43AE4206D1019800280ED110000C709D
:1030C000240A4C7003249BB20733A343D218009BFD
:1030D0009A42DED3FEBD4432F9E71000FAE7C0465B
:1030E000FC0F0000802213B503000324019189B274
:1030F000520107319B18A14304305A1A88235B05FB
:10310000C3181B68591C03D190429241104016BD50
:1031100099B2402907D80B000733A343C018904247
:10312000ECD30020F3E74430F9E7134B134A1B6854
:10313000126810B5FA24934201D81A00F824104BF3
:10314000E4021B689A4210D813000E4A12689A4291
:103150000ED3013307D1F823DB029C4203D10A4985
:10316000054808F045F8200010BDFC24E402ECE717
:10317000FE24E402F7E7C04600C0071100D00711A3
:1031800000E0071100F00711FFFFFF7FF0B59BB0D3
:10319000150004900391402A00D9A0E006AB5980A5
:1031A0001A80FFF7C2FF0400042816D9002206A9DE
:1031B000FFF768FF052810D906AB1B88AB420CD17E
:1031C000002D07D0514B2A000499C01808F000F9CF
:1031D000002802D101201BB0F0BD06AB1D802000ED
:1031E0000699FFF77FFF041E7BD1069B0793FFF72D
:1031F0009CFF80235B01C618802307001B039E42AF
:1032000001D3F826F60288235B05F31801931B68A7
:10321000013302D0019807F0ABFF3D49019807F058
:10322000E7FF3B1D0293331D05938822029B520545
:103230009B181B6808935A1C3CD044219AB20091F9
:10324000402A04D80320D11D814389B200910399FB
:103250001B0C8B4224D0402A22D80122300008A91E
:10326000FFF710FF021E1BD1380008A9FFF70AFF65
:103270000400042831D9009A059B9B188022520132
:10328000B218934240D288235B05C118009A09A85E
:1032900007F0D6FF1D4B009A09A9F01807F0F0FFC0
:1032A000009A029B9446634402931A4B029AFB18BD
:1032B0009A42BAD388235B05FC182168019801392A
:1032C00007F096FF200007F053FF039A07AB5A80E0
:1032D00030000799FFF706FF0400002C03D10020FF
:1032E00079E70428FBD988235B05E018069907F0E5
:1032F0007FFF0323EA1C9A4300D16BE7034B049939
:10330000E01807F0BDFF65E70424ECE704000011B6
:10331000FFFFFF7FF80F0000F7B505001400402AFB
:1033200021D8002701AE71803780FFF7FEFE042808
:1033300016D93A003100FFF7A5FE042810D93688C7
:10334000BC420BD0BD4209D0221CB44200D9321C71
:10335000064B92B2C118280007F072FF30B2FEBDD2
:10336000C04300B2FBE703204042F8E7040000112D
:1033700037B5042204000D0001A81649FFF7CCFF61
:10338000020004280BD1019BA34208D3AB4204D016
:10339000104901A80195FFF7F9FE01203EBD0E4C32
:1033A00023682000019307F0E3FE01992000013912
:1033B000019107F01DFF80235B01E418074B9C423D
:1033C000EED10422034901A80195FFF7DFFE00209A
:1033D000E4E7C0465555000000C007110000081181
:1033E00030B589B007F0FCFC102269461E4807F092
:1033F000AFFE1E4B009A9A4205D1019B0F2B2FD98D
:10340000029B013301D100230293029B002B03D0C6
:10341000049304984168084709B030BD1034102265
:10342000200004A907F094FE029B013301D1069B02
:103430000293882304995B05C918059B06981A0313
:10344000120B04910592814203D02B4201D107F067
:103450002FFF019B013B0193019B002BDED1CFE7A6
:10346000E025014C2D03F7E70000011150485936C3
:10347000F7B50F490F4B0A6804001A4084235B001C
:1034800013430B60030003271033019300252E0024
:10349000112007F0CDFD084B1B683B40AB400235C7
:1034A0001E43202DF4D1019B40C4A342EED1F7BDB1
:1034B0005CF0004000FEFEFF64F00040802270B52A
:1034C000AD4CAE4BD200002120001C6007F080FE06
:1034D0002300AB4A88331A60AA4B1A786E23002A5D
:1034E00000D01133E3620A232365A74B1878A74B5A
:1034F000A0630138E361C3B2032B01D81023236218
:10350000A34B37226361C823DB00A36123008C3304
:103510001A60082336210F3AE518E16323646264D8
:10352000E9670439251DE96725003B26BC352E6077
:103530002500C0352B602500C4352A6025000636DD
:10354000CC352E602500083EC8352E602500D035CC
:1035500029602100D4310B602100D8310A6021009C
:103560000225E0310D6025004221DC35296025006F
:103570001B3EE4352E602500E8352B602500EC3538
:103580002A6022000525F43215602200F032116015
:10359000220018319032116022009432136023000F
:1035A0003C2298331A60AF23DB002360794B2363FE
:1035B000032805D807F024FF33023537152363604D
:1035C00096232100FA225B00A360E360C8332361E5
:1035D000714BFC319200A3640A6062626F4A704DC5
:1035E000A2627322E2656D3A6265A2650232E56409
:1035F0004A600221616696218900A16662670921FD
:103600000022E166A2676749674A684E2167E26760
:103610003560032811D807F0F3FE96089EA6102304
:10362000CDE70E23CBE70C23C9E720001A259C30F9
:10363000056020000735A03005602000A830036039
:103640002300FA20F8338000186023006420A4339C
:10365000186023005F38AC33186023000338B033A0
:1036600018602300C630B433186023000020B8333C
:10367000186023003825FC339D604D4D5A665D640B
:103680004C4D9A64DD619625AD001D624A4D9A67E6
:103690005D62F53DFF3D9D621E25484ADD66186767
:1036A0005867D9651966DA67BE23C021444A5B00B2
:1036B000E250444B4900635004316250C42252002E
:1036C000A350FA23E4205B000432A3500432A35039
:1036D0003D493E4A3E4BD1603E49800019503E492B
:1036E000E938FF3819503D49043019503C49103829
:1036F000D1613C4911633C4951633C4911603C49EB
:10370000195019003B48F83108603B49D1658221C6
:103710003A4A89005A501A0039490832D1671A00CA
:103720003849B43211608821374A89005A501A004A
:10373000364988321160364ADA6407F0C9FC012044
:1037400007F0EEFD70BD200014259C3005602000C0
:103750000435A03070E7200010259C300560200063
:103760000335A03068E720000E259C30056020005E
:103770000235A03060E7C0460004FF1FB065FF1FA0
:10378000A070FF1F8845FF1F4A0AFF1F3A0700006D
:1037900080C3C9019A02000050C300006A180000EB
:1037A000280A0000204E000088130000F009FF1FC7
:1037B0000040001168100000C4090000DC05000092
:1037C00040420F0010270000FD1BFF1FFC00FF1FE1
:1037D0000000FF1F252FFF1F4D32FF1FE530FF1F89
:1037E000D91FFF1FF51FFF1FA121FF1F491FFF1F2B
:1037F000C528FF1F8D2CFF1FD918FF1FD127FF1FC2
:103800003925FF1F4525FF1F491EFF1F011FFF1FF1
:10381000C11DFF1FF7B50B0CFF27012200930023EA
:103820003C001E001D009446019089B262469A40F9
:103830001000084018413618B6B2FF2F02D1012EF1
:1038400000D19FB2009802401A41AD18ADB2FF2CD2
:1038500002D1012D00D19CB20133102BE6D10320FF
:10386000012E07D1012D04D1019B2401E4191C7004
:103870000138FEBD102EFCD10238102DF9D00230D7
:10388000F7E710B5064C2378002B07D10548FFF762
:10389000EFFD0548FFF7ECFD0123237010BDC04686
:1038A0007065FF1F8465FF1F7465FF1FF0B58BB047
:1038B0000D0001230190102936D8FFF7E2FF002305
:1038C0001A001B48C15C01335218102BFAD1023B7D
:1038D000002A29D0174B184C1F68002306A9E25C68
:1038E0001600FA5C56405E540133102BF7D102AA41
:1038F00007F096FB2A0002A9019807F0D9FC07F00F
:10390000DFFB23681B18236007F0DAFB63681B18D2
:10391000636007F0D5FBA3681B18A36007F0D0FB1A
:10392000E3681B18E360002318000BB0F0BDC0462D
:103930008465FF1F2844FF1F7465FF1FF0B5022335
:1039400001245A4E5A4D5B4F33702C703B688FB038
:10395000552B00D1A6E0042005F0F4FF002800D18B
:10396000A0E00023210000930420534A07F078FBD5
:103970008023DB059C62FFF733FD002006F07AFA16
:1039800007F0D6FCFFF79AFD07F052FD1F22012435
:1039900000214A4B0EAF1A70494B1C70494B1970ED
:1039A000494B19689143163A0A431A606022196814
:1039B0009143403A0A431A6007F02AFD07F020FBC2
:1039C000C120FF21414B80001A588A431A50C5225A
:1039D000920098588843BF390143995098583C4900
:1039E00008408021C9010143802099509958C005A1
:1039F0000902090A0143995080213648490107F01C
:103A000057FA03232200344901940093334807F006
:103A10000FFA2C22324903A807F012FC03AC61789C
:103A20002078023405F0B4FFA742F8D1002111201C
:103A300006F0C8F82B4B2C4A196803201140A0222D
:103A4000D2020A431A608022196892040A431A605B
:103A50001968264A1140802292030A431A60244BB7
:103A6000244A934200D8012007F092FB07F090FC13
:103A700007F056FA307807F02BFA2878C0B207F032
:103A8000E7FA07F05DFB0C49042007F0E9FB06F0BC
:103A9000BDF900F0A3F800F007FD00F005FA0020E2
:103AA0000FB0F0BD00233B6067E7C0464A0AFF1F26
:103AB0008845FF1F34F000403B000108480AFF1F03
:103AC000490AFF1F680AFF1FBCF0004000E100E048
:103AD000FF00FFFF8C45FF1F1058FF1F8C55FF1F75
:103AE00060B4001114F00040FF7FF8FFFFFF9FFF5C
:103AF000A070FF1F0080FF1F70B500252849294ACC
:103B000029484D6308CA1B051B0DED188242F9D1E7
:103B10000022264B8B63264B08211A628022254BFC
:103B20009205DA67244BDA688A43DA60234A12780E
:103B3000012A03D09A6822490A409A600121EE24A2
:103B40002048E40002686C438A430260DA6811206E
:103B50008A43DA6007F0FCFB112007F089FB112093
:103B600007F06EFC184A200C0400642390420AD827
:103B7000FA220023D200904205D9144B0A21C01822
:103B800007F006FAC3B2124A1372124BD4801B78A4
:103B9000002B04D1104B1021187807F0C9FA70BD22
:103BA000000005408805054000060540FF010000B3
:103BB00000F0004004E100E03CF000404A0AFF1F32
:103BC000FFDFFFFF00380040B70B000030F8FFFFB9
:103BD0000863FF1F2C65FF1F2063FF1F002210B525
:103BE0001100112007F05CFA10BD0000F8B50023A9
:103BF00001250826344F354C3B62E3681120AB4366
:103C0000E360E368B343E36007F032FB112007F0A1
:103C10009FFB112007F054F9402322681120134321
:103C2000236080236268DB02134363608023A26801
:103C30001343A360A368264A1340A3608023A268AD
:103C40009B0113431022A360236C93432364236CD2
:103C50002B43236480235B003B62226B1D4B1A4085
:103C60002263626B1A406263A26B1A40A263E26B2A
:103C70001340E363E368184A1340184AE36013688B
:103C80002B43136007F0C4F8FD21154B154A89003A
:103C90005A508023C720626B5B0313436363E3685E
:103CA00080003343E360E3680F4A1D430F4BE56038
:103CB00019581140802212020A431A50802292059C
:103CC0001A600B4B5E63F8BD00F000403CF0004012
:103CD000FFFFDFFFEFFFEFFFFFFF7FFF0038004038
:103CE0000000FF1FF93A0011FF00FFFF00E100E0B4
:103CF0000000054030B503A804880B20002C0ED12D
:103D00004968074D08784978090201430A20A94209
:103D100005D1012120001980024B1B7A137030BDA0
:103D2000192A00000863FF1FF7B5150008AA1688B6
:103D30004A680F4F14785278120222430A24BA427A
:103D400014D10122DBB2019200962A0006F0AEFFE8
:103D5000041E0BD1074B1B68002B07D068782A780C
:103D60000002104342425041013098472000FEBDFE
:103D7000022900009062FF1F30B50125037904007D
:103D8000BFB02B4212D00A49408806F0FBFA284205
:103D90000CD06A46074B69465B8D55801380064BF5
:103DA00060881B7A1371002203F0AEFB3FB030BD78
:103DB0008862FF1FD041FF1F0863FF1F10B5054930
:103DC000054806F095FA0421044A054806F052FA1F
:103DD00010BDC0468862FF1FFFFF00008CB40011B9
:103DE000D041FF1F10B5024804F014FA10BDC046C0
:103DF000793D00110623837010330371443B4371F6
:103E00002A3383714433C37100230222012110B588
:103E100003720E4B027041701C8881724472197AD1
:103E20000273C1729A784273DA7882730322C27382
:103E30001A7902745A7942740C2282749A79C27483
:103E4000DB7903751123C37010BDC0460863FF1FE3
:103E500010B5142007F054F9124B142200211860F9
:103E600007F016F9002007F0F3F9012007F000F938
:103E7000022007F085F9032003F070FC042005F010
:103E800085FC052002F0BEFE062003F07BFB072028
:103E900000F018FF082006F0CDF9092000F02EFDF3
:103EA00010BDC0469462FF1F10B507F029F801202D
:103EB00007F0B6F906F08CFF002010BD094B10B5D5
:103EC0000400984205D0012904D12000064906F0DB
:103ED0000FFA10BD0229FCD1013904F059F900286C
:103EE000F3D0F6E7FEFF0000BA62FF1F70B50D7A4F
:103EF000100004AA2C00168810221440154220D16C
:103F0000002E20D10A78022A18D14A6851781578F3
:103F10000E4A09022943914205D00D4A914209D027
:103F20001C800A2404E014220A491A8007F0C0F910
:103F3000200070BD0C2208491A80F7E71C8001247C
:103F4000F6E70824F4E70B24F2E7C046F3FF00008D
:103F5000F4FF00000C44FF1F50B5001110B5040021
:103F60000749084806F0C4F9074804F093F8002010
:103F7000E40704D50721054A054806F07BF910BD82
:103F8000BA62FF1FFFFF0000BD3E0011D0B4001158
:103F90001442FF1F00B5BFB06A460B4B0B491B888C
:103FA00001A813800A4B1A7800F0B2FA6B4680B26F
:103FB0005880002805D0074B00226946188803F076
:103FC000A3FA3FB000BDC0466E42FF1F9962FF1FBB
:103FD0009862FF1F6E43FF1F00B5BFB06A460B4BD0
:103FE0000B495B8D01A813800A4B1A7801F0E4F9A4
:103FF0006B4680B25880002805D0074B00226946E6
:10400000188803F081FA3FB000BDC0461442FF1F7C
:10401000C362FF1FC262FF1F6E43FF1FF7B50E0092
:10402000377A1C0008AB11003D001A8820231D4080
:104030001F423CD13378022B3BD173681F785B78E9
:104040001B023B431E4FBB4208D01E4FBB4214D045
:104050001D4DAB4221D00A252800FEBD002A2AD1E1
:10406000142C2AD82200F06807F022F9174B1C7094
:10407000012CF1D9FFF7B0FFEEE7002A1BD1202C6D
:104080001BD82200F06807F013F9114B04211C70B3
:10409000104B187807F04CF8DEE7E3B201240092E9
:1040A00001940A00310006F001FE0500D4E708255E
:1040B000D2E70125D0E70B25CEE70D25CCE7C0469A
:1040C000F3FF0000F4FF000002290000C262FF1F9E
:1040D0009862FF1F2063FF1F70B5160004AA1488A2
:1040E00005AA15784A685078117800022A4A0843D0
:1040F000801805284BD807F083F903131E29343F95
:104100000720032C0BD80422121BAA4200D92A0034
:1041100022491A803000091907F0CAF8002070BD42
:104120000720112CFBD81222121BAA4200D92A0008
:104130001B491A80EEE707200E2CF0D80F22121B25
:10414000AA4200D92A0017491A80E3E70720032C66
:10415000E5D80422121BAA4200D92A0012491A806B
:10416000D8E70720032CDAD80422121BAA4200D970
:104170002A000E491A80CDE70720032CCFD804224D
:10418000121BAA4200D92A0009491A80C2E700225C
:104190000A201A80C3E7C046DCD5FFFF1BB500111B
:1041A000E062FF1F0BB5001106B5001101B500114B
:1041B000FCB4001110B50D21024A034806F05AF86C
:1041C00010BDC046F0B400118442FF1F10B500219D
:1041D0000D2005F033FD01210C2005F02FFD06F028
:1041E000B7FE0400092006F06BFE0022184BDA66C9
:1041F00061321A6019685B3A9143023A0A431A60C5
:10420000144A944209D10A22DA6107321A62002262
:104210001A639A630132DA6310BD0F4A944203D1E4
:104220001E22DA610532F1E70C4A944203D13022B2
:10423000DA610632EAE70A4A944203D14322DA619C
:104240000832E3E7074A9442E1D16922F7E7C04622
:10425000005000400024F4000048E801006CDC023B
:104260000090D00300D8B80510B50024064B0920F3
:10427000DC6606F0FDFF21000D2005F073FC210037
:104280000C2005F06FFC10BD00500040F8B51C007C
:104290000023134D0F00EB666860160006F0A0FDCA
:1042A00001238022EB6623002F615200013B08D2DC
:1042B00006F086FF08200B4A1168002C03D120006D
:1042C000F8BD2A61F2E72B6F034203D02B69013C52
:1042D0003370013613685B1A012BEED90124EEE727
:1042E000005000406008FF1F002370B50C4C0D000B
:1042F000E366606006F074FD0123E366256106F065
:104300005FFF8020074A80001168636B034205D17C
:1043100013685B1A012BF8D9012070BD0020FCE75F
:10432000005000406008FF1F002370B5134C0E00C2
:10433000E3666060150006F053FD0123E366266125
:104340000F33626B1A42FCD02B0A23611023626B7D
:104350001A42FCD0EDB2256106F032FF8020084AF7
:1043600080001168636B034205D113685B1A012B4F
:10437000F8D9012070BD0020FCE7C0460050004085
:104380006008FF1F37B5204D2B7C002B37D0FFF77F
:104390001DFF0223002101AA287CFFF777FF6A4650
:1043A000040002230121287C0632FFF76FFF04433B
:1043B000FFF75AFF002C22D16B469A882B68D2BA9D
:1043C00053432A8911491B149B184B806B46DA888A
:1043D0006B6852BA5204520C53436A891B0C9B18E7
:1043E0000B481A1C1BB2834200DD021C130400D5CB
:1043F00000220B888A8001330B8020003EBDFEF72F
:10440000FFFD0124F9E7C046F462FF1F0863FF1FA8
:104410000F27000010B51B4B1A793F2A01D93F2204
:104420001A711979184A194811701822184902800E
:1044300018480A8002804A809A79174880240280AE
:104440000C208A80013242432401101CA24200D970
:10445000201C124AC88010805A79002A01D10132EA
:104460005A711A7A002A01D101321A725A791B7ACA
:104470000B4853430A21584306F08AFD094C20603B
:1044800010BDC0461463FF1F480AFF1F6C43FF1F87
:104490003445FF1F6A43FF1FF864FF1F6843FF1F77
:1044A000710200002463FF1F10B506210020FEF7F3
:1044B0005FFF124C002807D10C222000104906F0A3
:1044C000F7FEFFF7A7FF10BD0C2220000D49FEF7F5
:1044D00023FF0C2804D00C222000094906F0E8FE36
:1044E000094C0C2220000949FEF716FF0C28E8D0E1
:1044F0000C220021200006F0CBFDE2E71463FF1F31
:1045000044B50011FC0C0000F462FF1FF50C000024
:10451000F0B504000D00160085B0002A00D1C5E0FA
:104520000878002120706170262800D18BE00CD81B
:10453000072805D806F064FF4D28282828A099925E
:10454000252868D0FF236370A5E0712800D19AE088
:1045500014D8552845D05628F4D17A4D0C227A49E2
:10456000280006F0A5FEFFF755FF0C22774928002A
:10457000FEF70CFE0C222900601C46E0722800D1D8
:104580008BE0DC2800D193E0DB2800D0ADE0042EE6
:10459000D8D9AA786B7812021A43EB7810271B043B
:1045A00013432A7912061A430192052E05D0771F6C
:1045B0003A000198691D06F07BFE052229002000C3
:1045C00006F076FE3A000199601D06F071FE781D36
:1045D00005E00C2220005E4906F06AFE0C2005B0C2
:1045E000F0BD013A574E0C2A13D8002A0AD0691C94
:1045F000300006F05DFEFFF70DFF0C22300053493E
:10460000FEF7C4FD0C223100601C06F051FE0D20A7
:10461000E5E70C22EBE7013A4E4E0C2A11D8002AAE
:1046200008D0691C300006F043FE0C2230004A49D5
:10463000FEF7ACFD11223100601C06F039FE12209D
:10464000CDE70C22EDE7434D1122280006F020FDB6
:10465000FEF7D6FC11222900601CEEE712223F492A
:10466000601C06F025FE1320B9E708223C49601CB7
:1046700006F01EFE0920B2E705223A49601C06F04A
:1046800017FE0620ABE76978F72900D95AE7364BC1
:10469000188801F0EFFA0220A1E700F0FFFA012EDE
:1046A00002D06A78314B1A6006F0A2FE002096E72D
:1046B000022A00D846E76B786370AB78A3706F78F6
:1046C0001B021F43032A05D0033E3900B2B2E81C87
:1046D000FEF75CFD10223900E01CFEF71DFE030012
:1046E0000330002B00DB7AE72DE7DA2800D029E73A
:1046F000042E00D826E7AB786A781B021343EA78C9
:1047000012041A432B791B061343082E16D9AA79D3
:10471000697912020A43E979090411432A7A1206D7
:104720000A4303921A601B680522290020000393A4
:1047300006F0BEFD0422601D03A999E7FE22627007
:10474000F1E7C0461463FF1F44B50011FC0C0000E4
:1047500050B50011F462FF1FF50C0000E062FF1F6E
:10476000A844FF1F0063FF1F6E43FF1F34F000408B
:1047700070470000013870B5042809D806F040FEE3
:10478000030921081200144B0221187806F0D0FC0E
:1047900070BD114B0821187806F08AFC00220F4BDF
:1047A0001A71F5E700240D4B0B4D082128781A6883
:1047B0001C719C7106F08CFD2100287806F0F0FD3C
:1047C000E6E70123054C0821A371034B187806F096
:1047D0006FFC00232371DBE72063FF1F2463FF1FAF
:1047E00010B5002902D1112005F0ECF910BD000030
:1047F00010B5084B084C9881D881188258822078CF
:1048000002F09EF80422054B012120781A7006F070
:104810008FFC10BD3244FF1F5A65FF1F5965FF1FF3
:1048200010B501290CD11322064B11209A7105F005
:10483000C9F9054B1B78002B02D00448FFF7D8FFBD
:1048400010BDC0462463FF1F2C65FF1FC409000074
:104850000300F0B50A4D8E18B14202D15200801803
:10486000F0BD0C782F6824093C5D0F271C700C7874
:1048700001313C402F683C5D5C700233ECE7C04680
:104880006443FF1F10B5064A0649042005F09CFA50
:10489000112005F083FA0021112005F093F910BDD5
:1048A000E14700112148001110B5114B1A7818701A
:1048B000002A0ED000280BD10E4B1A78062A07D8F2
:1048C0005423D340DB0703D50B4B187802F038F89C
:1048D00010BD0028FCD0074B1B78012B02D0033BF6
:1048E000022BF5D8044B0121187806F021FCEFE7E4
:1048F0002C65FF1F5965FF1F5A65FF1FF7B5504D07
:104900002D242870FFF7BEFFFEF77AFB06F050FD5E
:1049100003224C494C48FFF79BFF030004221C7004
:104920004A490130FFF794FF30230222047043709C
:104930008370474C474B2000DA8706F059FA02286B
:1049400015D0062220004449FEF7E6FC06280ED0CA
:104950000321200006F064FD8D23E3706E3B23717C
:104960000622193320003C496371FEF70FFC0D232A
:104970003A4F3B4C3B4E3B70013B23700422033BC0
:10498000300039496370019606F092FC2D23012214
:1049900036493748A371FFF75BFF01223549FFF71E
:1049A00057FF01222A49FFF753FF0020FFF77CFF42
:1049B000314E324A30780121314B127801F082FFBA
:1049C0003A78012723003078002101F07BFF21781D
:1049D0002C4B0139019AC9B200201F7005F068FB09
:1049E000FA221C4B52019A81DA811A825A822021C2
:1049F000287806F0F5FC0120404205F0A5FB0120D7
:104A0000404205F041FCFFF7D5FBFFF7D7F900F076
:104A10006BFC01204042FFF7A1FA380006F000FAD3
:104A2000F72001F00BF93900287806F081FB28788F
:104A300002F0E2F8144806F0D3FAFFF7D7F8F7BD12
:104A40002063FF1FA844FF1FE062FF1F0063FF1FDA
:104A50006509FF1F3244FF1FADAC00002865FF1F32
:104A60000965FF1F0B65FF1F1BB500116709FF1FBD
:104A70001065FF1F6609FF1F5A65FF1F9643FF1F42
:104A80007743FF1FFA64FF1F2C63FF1FF8B50A006E
:104A900020230D001A40194232D0404B1B78002BC6
:104AA0002BD03F4C3F4E23790133DBB22371327A56
:104AB0009A4215D800272771FFF764FC6379013308
:104AC000DBB26371727A9A4202D86771FFF78EF88F
:104AD000354F3800FFF78EF93900152006F008FC35
:104AE000A379002B09D0013BDBB2A371002B04D1C9
:104AF000707964335843FFF77BFE20206840F8BD8F
:104B00000BB2002B0ADA294B187806F031FA00288C
:104B100001D006F045FA80200002EFE702240E00E3
:104B20002640214206D01E4B01201A71FFF7BCFE21
:104B30002000E3E70B0711D5FFF724FC00F0EEFBA4
:104B4000174A184953790133DBB25371497A9942B4
:104B500002D85671FFF74AF80820CFE71024214207
:104B600006D00E4B1B78002BE2D1FFF73BF9DFE7B5
:104B70000124214209D00E4800F068F806F078F9C7
:104B80002100112005F01EF8D2E70424080020407F
:104B90002142B4D0FFF7FEF9CAE7C0462C65FF1FDB
:104BA0002463FF1F1463FF1F7743FF1F2063FF1F52
:104BB0005C43FF1FF0B51B4B1B4F1B883A8804005A
:104BC0001A4E1B4D85B09A420DD832889A420AD3AC
:104BD000184B1A882B889A4205D1174A174B12880E
:104BE0001B889A421BD0052001F07EF83B8802AA60
:104BF00013803388019053802B88114D93800F4B85
:104C000002A91B88D3800F4B2A78188802F08AFDEE
:104C10000D4B08212878019A1C7006F019F905B08F
:104C2000F0BDC046F664FF1F6C43FF1F6A43FF1FC1
:104C3000F864FF1FF464FF1FF264FF1F6843FF1F47
:104C40005A65FF1F6E43FF1FF064FF1F13B50C4B27
:104C50001C78002C11D1002801D00A4B18600A4A98
:104C60000A4B11780A4A10780A4A01920A4A0092BD
:104C7000002205F015F9200016BD1124FBE7C046FF
:104C80005965FF1FEC64FF1F5865FF1F4865FF1F34
:104C90005A65FF1F3465FF1F3865FF1F10B5064BAF
:104CA00012201B78052B06D1044B13221988044BC4
:104CB000187801F0F5F910BD5965FF1F6E43FF1F0D
:104CC0005A65FF1F10B500240122114B5242187083
:104CD000104B1C70104B1A8001F08EFF04220F4BFA
:104CE00021001A700E480C3206F0D2F91022210071
:104CF0000C4806F0CDF907220B4B1C600B4B1C70C7
:104D00000B4B1C700B4B1A700B4B1C7010BDC0462C
:104D10005A65FF1F5965FF1F6E43FF1F5865FF1F30
:104D20004865FF1F3865FF1F3465FF1F0865FF1FBB
:104D30000765FF1F7043FF1F0665FF1FF8B5174C7F
:104D40000600257806A814240078052D23D1B41F69
:104D5000134FA5B21824BD421DD88D1FADB2BD4260
:104D600019D8FA256D00AA4215D21D000D4F0A3D33
:104D7000ADB2BD420FD80C4C26800C4C21800C49A2
:104D800000240A800B4A1380FFF714FF0A4B04210A
:104D9000187806F08DF92000F8BDC0465965FF1F50
:104DA000790C0000750C00006C43FF1F6A43FF1F65
:104DB000F864FF1F6843FF1F5A65FF1FF0B50BB271
:104DC0000D0089B0002B00DB76E1A64E307806F0AE
:104DD000CFF8041E55D00378A22B00D127E1D02BA9
:104DE0001AD0912B4AD143780E2B47D19E4B828803
:104DF0009A4243D19D4A83681278052A3ED1032006
:104E000018567F283AD09A4B1B68002B36D05B6827
:104E1000002B33D0984731E0807807282ED806F051
:104E2000EFFA042D1D444479ADDD6378002B11D1D8
:104E30000622E11C8F4806F03BFA01218B4B1970CA
:104E40008D4B1A78002A5BD08C4B307801F03AFDFC
:104E5000002855D00722854B1A7051E0617800294F
:104E6000F8D1E378002B11D0854A864B1278307840
:104E700001F028FD60706378002BEBD1200006F074
:104E80008FF880200002684009B0F0BD774B1B7896
:104E9000022BF3D00121307806F0CAF90028EAD1BC
:104EA0000121307806F044F9E5E76378002BD1D191
:104EB0006E4F032807D13B78052B02D101333B709D
:104EC0001EE00223FBE7704B1A88704B0293002A06
:104ED0000BD01B78002B03D00121307805F0B8FFF0
:104EE0003B78062B04D1013BE9E7029B1A70F7E7F8
:104EF000042B41D10121029B3078197006F018F97A
:104F00005B4B1B68002BB9D01B68002BB6D0574AEF
:104F100010787FE76378554F002B27D10622211D9B
:104F20005B4806F0C5F962895A4B5B491A80A28931
:104F30005A4B1A80E3890B800521397058490A8041
:104F4000584A1380228A584B1A80584B1B78012BE1
:104F500009D11F2000F0C8FEFA229200424304212A
:104F6000307805F075FF0022484B75E7312B00D0F3
:104F700070E70022454B1A700323A0E706220021A8
:104F8000434806F085F80023454A04211380454A2A
:104F900030781380444A138006F08AF8082130786C
:104FA00006F086F8A379083B5A4253412F4A03334F
:104FB0001370314B1B78002B06D0344B30781A78A5
:104FC000002A06D001F0BCFC0122324B52421A806A
:104FD00096E70121197006F0ABF8F5E70821307863
:104FE00006F066F86378002B00D047E72C4B2E4F75
:104FF0000293E388029A042113802A4B30780393AA
:105000002389039A138063893B8006F011F90028F5
:1050100000D033E7264B1B68002B00D12EE7039905
:1050200002983A88098800881B68984726E74379E0
:10503000132B00D022E70389012B0AD11D4B1B78CB
:10504000022B06D10821307806F032F8FFF726FE51
:1050500014E7052000F048FE08210200307805F032
:10506000F7FE0BE75A65FF1F051400005965FF1F87
:10507000EC64FF1F2D65FF1F9643FF1F7743FF1F43
:105080002865FF1F0965FF1F2A65FF1F2C65FF1F8D
:10509000FB64FF1F6E43FF1F0265FF1F0465FF1FB8
:1050A000F664FF1FF464FF1FF264FF1FFA64FF1F22
:1050B000E864FF1FF064FF1F8020C001014200D0A0
:1050C000E1E6CB0731D5324B1B78002B1DD0314E9A
:1050D00005AC3378052B1AD1023B23702E4B2100EF
:1050E0001B7823722D4B1B7863722D4B187801F0BF
:1050F0008DFB002809D007202A4B30701B68002B3D
:1051000003D01B68002B00D098470120BBE60E207F
:10511000254B06221B7825492370254B1B7863708D
:1051200002ABC01806F0C4F8D8E702230800184004
:10513000194209D0174B1B78052B03D11D4B18883A
:1051400006F0E6F802209EE60424214203D0FFF791
:1051500031FD200097E6082308001840194200D1CD
:1051600092E6154B1C78012C03D0022C0DD00820A0
:1051700089E6124B124A134913481B881288098882
:1051800000880094FFF7DAFDF1E7FFF787FDEEE70F
:105190002C65FF1F5965FF1F7043FF1F0665FF1F2A
:1051A0005A65FF1FEC64FF1F0865FF1F7143FF1F57
:1051B0000765FF1F6E43FF1FF064FF1F6843FF1F5B
:1051C000F864FF1F6A43FF1F6C43FF1F10B502A85E
:1051D00004880B20002C10D149680878497809020E
:1051E00001430C48814209D1022119800A4B598898
:1051F0001170DB7800205BB2537010BD074C0A20A1
:10520000A142FAD102211980034B998811705B7970
:10521000F0E7C0466E2A00000863FF1F6F2A0000F7
:10522000F7B5150008AA16884A680F4F1478527807
:10523000120222430A24BA4214D10122DBB20192A3
:1052400000962A0005F032FD041E0BD1074B1B68A7
:10525000002B07D068782A78000210434242504160
:10526000013098472000FEBD022900006C65FF1F39
:1052700030B5012503790400BFB02B4227D0154972
:10528000408805F07FF828420DD06A46124B6946E7
:105290005B8D138002235380104B5B889380608862
:1052A000002202F031F90E49608805F06BF8C00762
:1052B0000DD56A460B4B69461B8813800223538029
:1052C000064B9B8893806088002202F01DF93FB056
:1052D00030BDC0466465FF1F9843FF1F0863FF1F72
:1052E0005C65FF1FF243FF1F10B5074C0749200004
:1052F00004F0FEFF2000064904F0FAFF0721054AEA
:10530000054804F0B7FF10BDFFFF00006465FF1FF4
:105310005C65FF1FD0B500119843FF1F10B5024810
:1053200002F078FF10BDC046715200110200F0B5C6
:1053300001270A480A4E51188B1A002B00DCF0BDD9
:10534000082415784308684038404000805B013CE1
:1053500058406D08002CF5D10132EDE7FFFF000049
:10536000EAB50011F0B500250F269D4200DBF0BD27
:105370004C5D070944403440A400A05801357840F2
:10538000F3E70000F0B589B06A460D000B000F2767
:10539000110010351C780133260024093E40167098
:1053A00054700232AB42F5D12023024AFFF7DAFFF4
:1053B00009B0F0BDF0B50011F0B54D780B788BB0A9
:1053C0002D020C00170003901D43012A61D9964B52
:1053D0009D4200D877E001339D421CD1062A17D1A7
:1053E000CA788B7812021A430B791B0413434A794B
:1053F00012061A438D4B5A6100221A705A808C4A49
:105400005A608C4A9A608C4ADA6000200BB0F0BD7A
:1054100088225205EEE7894B9D423CD183498B7827
:10542000002B00D0F8E00C2A31D10F22A37893434F
:10543000E2781202134322791204134362791206AE
:1054400013434B60E279A07912020243207A0004F0
:105450001043627A12060243CA60E27AA07A12020C
:10546000024377484A81834208D804236F491422B3
:1054700003980B7005F01CFF1420C7E71201D21827
:1054800089235B059A42F0D801238B70BDE7022A7D
:10549000FAD00523EAE76B4A01239542E6D1FFF7EC
:1054A000FDFB052F0CD9E378A2781B021343227968
:1054B00012041A4363791B061343634A059313606E
:1054C00005F096FFA1E7594E3378002B9DD1B378B4
:1054D000002B00D1A2E0338901339BB29D4200D062
:1054E00095E0132AD5D9CF7C8B7C3F021221200076
:1054F0001F43FFF71BFFB84200D091E0002D41D1C0
:10550000E278A37812021A432379F1681B0413434B
:10551000627912061A4305920A23914213D1F53398
:10552000A370E370237163717389002B0AD1E37B4D
:10553000227C1B0212041343A27B134305931B0915
:10554000013373810023394E7289002A8DD0002BDC
:105550008CD1954266D270682F013818000B7369A0
:1055600000030590984205D9706105F001FEF378BB
:105570000133F37070681022A11C381805F080FE0A
:10558000358142E773890193013B9BB29D42D9D19A
:10559000E378A2781B0213432279776812041A4336
:1055A00063793E1D1B0613430593284B0422190003
:1055B00006A8029305F07CFE31000C2207A805F036
:1055C00077FE012006A94042FFF7DCFE019E10375E
:1055D000013E012E16D1154E059A0B2330618242F1
:1055E000B1D104220299706805F04AFE042205A98F
:1055F000706805F0E5FCF168059A08239142A2D194
:10560000F733A0E73900FFF7BDFE1037E0E79D4212
:1056100000D2FAE6072329E7022327E7032325E739
:10562000062323E7092321E7FFFE00000C44FF1FA8
:1056300000000111FFFF00005048593601FF000033
:10564000FFFF001102FF000034F000401844FF1F6C
:1056500010B5034C0B000122210000F06BFA10BDC5
:10566000115800110B8870B506000D000224162B8E
:1056700011D92B000322094900F05CFA041E0AD15B
:10568000074B2A881B88191C934200D9111C300033
:1056900089B200F0EFFA200070BDC0463D580011FD
:1056A000CA65FF1F10B54A780400013A0B000220BA
:1056B000012A07D80A78002A04D0052220000249CE
:1056C00000F038FA10BDC0466B5800110A7810B5CA
:1056D0000B0004000220002A04D007222000024907
:1056E00000F028FA10BDC046175900110A7810B50D
:1056F0000B0004000220002A04D0092220000249E5
:1057000000F018FA10BDC0467D59001110B5034CC9
:105710000B000B22210000F00DFA10BDAD59001155
:1057200010B5034C0B000D22210000F003FA10BD50
:105730001F5A001110B5034C0B000F22210000F07E
:10574000F9F910BD795A00110A7810B50B00040060
:105750000220002A04D011222000024900F0EAF9B8
:1057600010BDC046895A0011002310B5132219003C
:1057700000F0E0F910BD000010B5034C0B0017223B
:10578000210000F0D7F910BDDB5A0011002310B53D
:105790001922190000F0CEF910BD000010B5034C1D
:1057A0000B001B22210000F0C5F910BD155B001194
:1057B000F7B584890D0006000121002C22D00023BA
:1057C0008268D3561778002B1EDA0C2C1AD90C3CA1
:1057D000A4B2131940880093230002F076FE431E02
:1057E000984101307B06DB0F6B703F23013C1F406B
:1057F000A4B22870AF70AC80002C07D0B36801331E
:10580000AB6000210800FEBD0020EBE7AC60F8E7CC
:105810000B7803704B8843704B881B0A83700B799D
:10582000C370042070470420022B06D10020537857
:1058300011781B02009A0B43138070470B8803708A
:105840000B881B0A43700220704704200099834292
:105850000AD1537810781B0203430B80D3789078D9
:105860001B02034300204B807047F8B50D004B78B6
:1058700001240021461C03702B788B4201D82000A4
:10588000F8BD6B78B01C4F1C012B10D18900691832
:105890004B88022233704B88B9001B0A7370691859
:1058A00005F006FD04360434A4B2F9B2E4E712238D
:1058B00059436B185A88043132705B8810221B0AD6
:1058C0007370691805F0F4FC12361234ECE770B509
:1058D000049D14001E00052B01D8042070BD6378C0
:1058E00012781B0213432B80E378A2781B02134328
:1058F00002226B802A71211D681D063E05F0D8FC2E
:10590000B2B22A81F02AE8D82800A11D0A3005F099
:10591000CFFC0020E2E7002310B50A789A4201D8B4
:10592000900010BD9A008A1854880133047054887E
:10593000DBB2240A4470948884709288120AC27080
:105940000430EAE710B51100029C062B04D00420B5
:105950001022142B01D010BD022222714B7808783E
:105960001B0203432380CB7888781B0203436380A8
:105970000431601D05F09CFC0020ECE710B50C78AC
:105980008B7804315C43E4B203702200013005F0EF
:105990008FFC601C10BD0420022B06D10020537820
:1059A00011781B02009A0B431380704710B50C004E
:1059B0000A88023105F07CFC208810BD70B5040017
:1059C0000D0004981100012B01D8042070BD167839
:1059D00052781202324302800200F832557014707D
:1059E000E825002C00D10C35023B9AB24280AA4235
:1059F000EBD80231043005F05BFC0020E6E7042020
:105A0000009983420AD1537810781B0203430B801C
:105A1000D37890781B02034300204B80704710B569
:105A20000C000A88023105F043FC208810BD0000FC
:105A300070B501211E000420049C0E400B4218D1B9
:105A4000CB40DDB28D4214D90A49DBB209889942B4
:105A50000FD32300F6331D70330058001118497816
:105A6000165C0902314301332152D9B28D42F4D878
:105A7000002070BD2C44FF1F10B50C000A880231B5
:105A800005F016FC208810BD10B50C788B78043119
:105A90005C43E4B203702200013005F009FC601C95
:105AA00010BD10B511000298032B01D8042010BDC1
:105AB00014785278043B120222430280CA788C7810
:105AC0001202224342809AB28280F22AEED8043136
:105AD000063005F0EDFB0020E9E710B50C000B885F
:105AE00003700B881B0A43704B8883704B881B0A1A
:105AF000C3708A880430063105F0DAFBA0880430D0
:105B000080B210BD0420012B03D100201378009A2D
:105B10001370704710B50C000B8803700B881B0ABC
:105B200043704A880230043105F0C2FB60880230BD
:105B300080B210BDF0B589B003931E4B02924200B3
:105B40000700D05A019102F010F81325061E2DD03F
:105B5000029B01240370019B002B04D000190399C0
:105B60009847001984B26B461B7A5BB2002B0FDAA0
:105B70001021380002F00CFB1925002813D1300049
:105B80003219E1B202F056FC051E0CD10C34A4B25D
:105B9000042304AA380005A993800696948101F095
:105BA0009FFD051E02D0300005F07AFB280009B0E9
:105BB000F0BDC046C865FF1F70B505000C00002889
:105BC0000CD00020814209D010222000044905F0A9
:105BD0006FFB01202B7823736B78637370BDC04615
:105BE00030B60011F0B506000D0017001C0085B09E
:105BF00002291BD00020102907D1022B07D0102B1F
:105C000003D115E00020102C08D005B0F0BD694686
:105C10003800FFF7D1FF2A0069460BE069463000E3
:105C2000FFF7CAFF22006946380004E0022BE9D1E1
:105C30002A003900300005F053F9E6E7031CF72885
:105C400000D9F723032008499AB2013A0B80D317F1
:105C5000034006499B189B100B80D30F04499B18E7
:105C60005B100B807047C0463044FF1F2E44FF1F5F
:105C70002C44FF1F034B1B888B4202D3024B400076
:105C8000C15270473044FF1FC865FF1F014B4000E1
:105C9000185A7047C865FF1F1722014B1A807047BA
:105CA000C865FF1F70B505000E2005F029FB041E16
:105CB00013D0D02303700023062283700749457058
:105CC000033005F0F5FA064B2100DA8A62811B7E6B
:105CD0002373044B187805F093F870BDE465FF1F3B
:105CE000D465FF1F8044FF1F262803D8024B4000C5
:105CF000C05A70470148FCE73244FF1FFFFF000015
:105D000070B506000C00094D1C220021280005F08A
:105D1000BFF9074B1E70074B1C7005F0C1F801233B
:105D2000002801D0002312202B7070BDD465FF1F06
:105D30008044FF1FF565FF1F70B505000D4C08007E
:105D4000E260A16010220021656005F049FA012897
:105D500003D11021A06802F048FD10220021280084
:105D600005F03EFA012803D11021606802F03DFDE4
:105D700070BDC046D465FF1F70B5041E05D1002953
:105D800003D006220D4805F093FA0D4B1D78012D26
:105D900011D1002C05D102221A7005F0F1F828006B
:105DA00070BD00221A70074B1B78FF2BF7D0200024
:105DB000FFF778FFF3E70025F1E7C046E465FF1F32
:105DC000D465FF1F8044FF1F030010B5002801D1D8
:105DD000002010BD00780B4A002803D15988D182D9
:105DE0001B7913761378022BF2D10023984200D14D
:105DF00003331370044B1B78FF2B01D0FFF752FFC6
:105E00000120E6E7D465FF1F8044FF1F002911D061
:105E100000280CD04B79012803D140225242134371
:105E200003E03F221340032802D001204B7170474A
:105E30004022F4E70800FAE770B5094D0100287820
:105E400000280BD0074C0622200005F031FA210073
:105E50002878FFF7DBFF200005F032FA70BDC0465E
:105E6000F465FF1FCE65FF1F00290AD0012808D165
:105E70003F224B799343C02B03D0403B5A425341BE
:105E8000981C704770B5174D06002B78FF2B15D066
:105E90000A2005F035FA041E10D0D0230370C83B49
:105EA0008370114B11491B784670C3700622043071
:105EB00005F0FEF92100287804F0A2FF0C4B1B78B6
:105EC000012B0DD10B4B1B68002B03D09B68002BC3
:105ED00000D09847084B04211878084A05F0F8F9D3
:105EE00070BDC0468044FF1FF465FF1FCE65FF1FD5
:105EF000F065FF1F1C66FF1F2066FF1F60EA0000A1
:105F0000014B98687047C046D465FF1F014BDB68A2
:105F100018687047D465FF1F074B10B5DA6813681F
:105F200001331360054B1878FF2803D08021C90185
:105F300005F0FEF810BDC046D465FF1F8044FF1F6A
:105F4000F7B50E0002F0B8F8051E1CD00E4B066225
:105F50001F78002F00D10778AB791020019305F04E
:105F6000CFF9041E0FD0D0230380C73B8370019B61
:105F7000E91DC3700622043005F09AF921003800AB
:105F8000E66004F03DFFF7BD7E44FF1F014B18782B
:105F90007047C046F465FF1F054B002805D1054B2F
:105FA0001A78054B002A00D1014B18007047C046F3
:105FB000E465FF1FF465FF1FCE65FF1F014B5868A6
:105FC0007047C046D465FF1F024B1868431E9841B6
:105FD000C0B27047F865FF1F421E03000120152A5A
:105FE00003D9FF3B5A425341D8B27047F0B51C0069
:105FF00000230E0085B0039002920B70029A934228
:1060000001D3002019E0E55C5A1CD2B2002DF8D073
:10601000029851198142F4DC0233DFB2A35C18000C
:106020000193FFF7D9FF002807D0013D019A03999A
:10603000EBB233708A4202D1E01905B0F0BDDB1932
:10604000DBB2DBE710B50C0002F08EF80300122083
:10605000002B03D02100588805F01AF910BD00006C
:1060600070B50E4D84006359002B15D0186A0028B6
:1060700001D004F09DFF2B59586A002801D004F08C
:1060800097FF2B59986A002801D004F091FF2859F6
:1060900004F08EFF00232B5170BDC0460466FF1F25
:1060A0001C4B70B504000E00150099420AD11A4B22
:1060B0001B68002B01D1122070BD1B68002BFAD089
:1060C0009847F9E7154B994215D1134B1B68002BE4
:1060D0000AD01B68002B07D09847002804D1104B2A
:1060E0001C70104B1D70E7E729002000FFF7AAFF86
:1060F0000028E1D1F3E7080001F0DEFF0028DAD044
:1061000003780320A342D7D12900300005F0C0F85E
:10611000D2E7C046FEFF00000066FF1FFFFF000041
:10612000FD65FF1FFC65FF1FF7B50400808801F0C7
:10613000C3FF0025A84203D00578A08801F0F8FF2E
:106140001C4E3378002B1FD0AB421DD11A4B2800B8
:106150001978FFF777FF002818D000233370A37950
:106160000820A778A688019305F0CAF8011E0DD073
:10617000D0230370CA3B8370019B47708680837174
:10618000280004F03DFE01E0002DE8D1A0880B4B73
:106190008200D358002B01D0FFF762FF1721A0889F
:1061A000FFF768FDA08801F017FDA08801F0EEFD63
:1061B000F7BDC046FD65FF1FFC65FF1F0466FF1F9E
:1061C000F0B587B01D000CAB1B88070001930DAB29
:1061D0001B88142002930EAB1B88160003930FAB91
:1061E0001B880091049310AB1B88059305F088F879
:1061F000041E1AD0D0230370CB3B47708370C67047
:10620000062229000430002D11D005F051F8019B21
:1062100021006381029B0098A381039BE381049B7F
:106220002382059BA37404F0EBFD07B0F0BD04F0DE
:106230002FFFECE7F7B5009308AB1B8807000C2095
:106240000D001600019305F05BF8041E13D0280022
:1062500001F032FF00280FD00078D0232370C93B13
:10626000A370009B21002381019B6770A580E680BD
:10627000638104F0C5FDF7BD014B1878EDE7C0461A
:106280008044FF1F13B5040064890389C288818894
:10629000C0780094FFF7CEFF13BD000010B5044C8A
:1062A0002068002803D004F083FE0023236010BD83
:1062B0000866FF1FA122F0B5818892004A43384B3F
:1062C000384F1B6804009B189D2292009B1882790E
:1062D00089B01A603B68002B5FD01D78324B1B6879
:1062E000002B04D05B68002B01D0002098472600CB
:1062F00008363100E079FFF7B7FD237DE071020039
:10630000E0780493638A29000393238A0293E38944
:106310000193A38800933300FFF752FFE378002B2B
:106320000BD1E289A379A18802920196E279280033
:106330000092012201F0CAFEE0703B68002B20D0E1
:10634000FFF7ACFF194D287800281AD0184B1978A0
:10635000FFF778FE002814D02B78E6780820079302
:10636000A78804F0CDFF011E09D0D0230370CA3BDB
:106370004670837087808671079804F041FD002382
:106380002B701721A088FFF775FCA08801F024FC72
:10639000A08801F0FBFC09B0F0BD064B9DE7C046AC
:1063A0003409FF1F0866FF1F1C66FF1FFD65FF1FE6
:1063B000FC65FF1F8044FF1FF8B5070008000E00B2
:1063C00001F07AFE041E18D02620FFF78DFC051E72
:1063D00000D12578062004F093FF041E0DD0002183
:1063E000062204F055FED0232370C23B21006770C3
:1063F000A370A680E8B204F003FDF8BDF0B585B047
:1064000001930AAB1B78070002930BAB1B780800C3
:106410000D000092039301F04FFE061E22D01020C3
:1064200004F06EFF041E1DD01022002104F030FE87
:106430002620FFF759FC002800D13078D0232370A4
:10644000C13BA370009B21002372019B67706372A4
:10645000029BA580A372039BC0B2E3720C9BE36016
:1064600004F0CEFC05B0F0BDF7B50D00019001F0D1
:1064700023FE071E20D00E2004F042FF041E1BD076
:106480002620FFF731FC061E00D13E78D023238062
:10649000C53B0622A370F91DE01C04F009FF019B17
:1064A0002A0063810123DD401A401D402100227330
:1064B0006573F0B204F0A4FCF7BD0000F0B585B040
:1064C000029010000D0017000A9E039301F0F4FDE6
:1064D000041E31D0029B002B2ED1039B02795B0757
:1064E00024D5122313430422002E08D10B9900292E
:1064F00005D10C99002902D10D9900291AD01A430F
:106500000D9B2271002B00D0C9E0002E00D1CFE0FE
:10651000002D00D0CCE0606A002801D004F048FDD6
:106520001C21300004F00CFD606205E002239A4358
:106530000E33D7E793432371654BBA00D458002C30
:1065400000D1AAE0002E10D0236A002B03D11C201A
:1065500004F0D6FD20625E4BBA00D358186A0028BA
:1065600003D01C22310004F0A3FE0C9B002B12D0A0
:10657000574CBB001D596B6A002B03D1162004F049
:10658000BFFD6862BB00E358586A002803D016229A
:106590000C9904F08DFE0D9B002B11D04C4DBC00CE
:1065A0006659B36A002B03D1142004F0A9FDB06230
:1065B0002B59986A002803D014220D9904F078FE14
:1065C000380001F079FD051E67D0414BBA00D35861
:1065D000002B62D01A6A3420002A00D11C389A6A33
:1065E000002A01D0143080B20B9A002A01D01C304E
:1065F00080B25B6A002B01D0163080B204F080FEBE
:10660000041E4AD01822002104F042FD2620FFF784
:106610006BFB0190002801D12B780193D0232370CC
:10662000029B200063700A23294EA370039BBD00C8
:10663000A371AB59A780196A1830002905D01C2214
:10664000A06004F035FE200034307359996A0029A7
:1066500007D0030014221433E060029304F028FEF4
:1066600002980B9B002B08D003001C221C330B99B3
:106670002061029304F01CFE02987359596A0029A4
:1066800003D01622606104F013FE6B4621001879D6
:1066900004F0B6FB3800FFF7E3FC05B0F0BD1022B4
:1066A0000D9B0D991B69A018236204F001FE2CE7D5
:1066B0000B9B002B00D13FE7012D00D03CE7606A27
:1066C000002801D004F074FC1C210B982AE7C04676
:1066D0000466FF1F10B5044C2068002803D004F0A6
:1066E00067FC0023236010BDF865FF1F0B4B07B547
:1066F0001A68002A01D100200EBD6946531C0120F2
:1067000012780731FFF772FC0028F4D002780123D9
:10671000100018401A42EED0EEE7C0461466FF1F84
:10672000F0B51F4F01203B6887B0002B25D09B7828
:10673000059300F0B3FB002821D00A20FFF7D4FA1C
:1067400004000B20FFF7D0FA164B05001E78731ECD
:106750009E413B68F6B2191DD878FFF757FB3B689E
:106760002900DA7A043303929A7901930292009015
:1067700033002000059A04F063FC07B0F0BDFFF77A
:10678000B5FF002805D00620FFF7AEFA0400072069
:10679000D8E70820FFF7A8FA04000920D2E7C0468E
:1067A000F865FF1FF465FF1F70B50A4E04003378CB
:1067B0000D00FF2B0DD0042004F0A2FD011E08D017
:1067C000D0230370CE3B45708370C470307804F0E2
:1067D00017FB70BD9044FF1F70B5040006200D002C
:1067E00004F08EFD011E0AD0D0230370CD3B8370D0
:1067F000054B44701B688580187804F001FB002C61
:1068000001D0FFF767FF70BDF865FF1FF8B5264F91
:1068100006003B680D001124002B05D10522234BF7
:106820001B78134202D112242000F8BD204A102404
:106830001268002AF8D01278002AF5D0DB0719D5A3
:106840002B789A1E012A1AD80C2004F059FC132424
:1068500038600028E8D000230A224370290006701F
:10686000023004F025FDFFF75BFF041E0AD0FFF79E
:1068700031FFD9E700F012FB0028E1D1E4E7002B5B
:10688000E2D0D0E70B4B1B78032BCDD11D20FFF7B7
:106890002BFA094B18800028C6D0084B0421187821
:1068A000074A04F015FDBFE7F865FF1FF565FF1FF8
:1068B0001466FF1FF465FF1FF265FF1F2066FF1FB0
:1068C00060EA0000F7B50193194B14001A7805230C
:1068D00006000F0012201A4221D0012920D1154BA9
:1068E0001D68002D1BD002201F2C18D8002C02D0B0
:1068F000019B002B13D0104B1F221E706E1C002119
:10690000300004F0C5FB01992200300004F0D0FCF7
:10691000310020002C70002F06D004F051FDFEBD88
:10692000064B12201D68DCE704F04AFAF7E7C04680
:10693000F565FF1F1466FF1F9044FF1F1066FF1FC1
:10694000F8B50F4E12243368002B17D01B780F3C7C
:10695000834213D100250B4F0221387804F0A8FBA5
:10696000094B042138781D8004F0A2FB074B280056
:106970001D8033685C7004F0BBFB04002000F8BD90
:10698000F865FF1F2066FF1F0C66FF1FF265FF1FE3
:1069900070B5012823D11B4C2388002B03D01A4A41
:1069A0001578002D07D0194B1B68002B02D01878E2
:1069B000FFF7C6FF70BD3B2B02D93C3B2380F9E7B4
:1069C000134E0221307804F073FBFA2223889200E0
:1069D00002215A43307804F03BFA2580EAE70B4B5A
:1069E0001B68002BE6D00B4B1B785B07E2D5084BEE
:1069F0000221187804F05CFB0022024B1A80FFF79A
:106A000069FED7E70C66FF1FF065FF1FF865FF1FE3
:106A10002066FF1FF565FF1FF8B51E4D286800288A
:106A200003D004F0C5FA00232B601B4E3068002809
:106A300003D004F0BDFA00233360184F05243B78DF
:106A400018002040234221D0154800F02BFA3B7853
:106A5000234213D0202004F053FB2860002813D0D9
:106A60002022002104F014FB202004F049FB041E26
:106A7000306005D02022002104F00AFB002004E051
:106A8000286804F095FA2C601320F8BD00F00AFA8B
:106A9000F4E7C0461466FF1F1066FF1FF565FF1F71
:106AA0008444FF1F10B50A4C23681A1E0ED000281C
:106AB00008D10130587004F01BFB002805D0236872
:106AC000002B02D00021FFF787FE0122100010BD2D
:106AD000F865FF1FF7B5274E050033680191181EB2
:106AE00021D05C78244F012C30D1FFF7FFFD002826
:106AF00025D02000FFF7F8F80400412814D91F4BD7
:106B0000022118781E4A04F0E3FB1E4B3C3C1C801B
:106B1000022233685A703B78002B14D12800019967
:106B2000FFF75AFE0120FEBDFA2292004243002ADE
:106B3000EED0124B0221187804F08AF9E8E7FFF74B
:106B4000D3F80200F3E700233B70EBE73B78002B20
:106B5000E8D1032004F0D4FB011E08D0D023037039
:106B6000CC3B457083703368187804F049F9FFF71F
:106B7000B1FDD7E7F865FF1FF065FF1F2066FF1F17
:106B800060EA00000C66FF1F10B5174983880200F9
:106B90008B4220D011D815498B4217D014490020C0
:106BA0005B1899B2012907D8926811785A4253416B
:106BB000D8B2FFF7F9FD012010BD0E4A00209B1846
:106BC00007229BB29A424041C0B2F5E78368187829
:106BD000FFF768FFF0E7836899785A780902187818
:106BE0001143FFF777FFE7E70A20000006200000C7
:106BF000F8DFFFFFAFDFFFFF014B18707047C046A3
:106C00009144FF1F10B5064C207001F031FA207836
:106C100004F026F90521207800F052FD10BDC04691
:106C20002066FF1F0BB273B50D00002B00DBC4E024
:106C3000884B187804F09CF9041E0ED00378912B31
:106C40000FD0A22B00D1A1E0834B1878FF2852D09F
:106C5000210004F0D5F800284DD1802000026840C2
:106C600076BD43780F2B76D013D8052B70D00E2B22
:106C7000EAD18088794B98422BD8794B98421BD81F
:106C8000784B9842E0D1A3681878591CFFF774F844
:106C900038E03E2BD8D18378032B74D06CD8012BED
:106CA0006ED0022BD0D1704B1B68002B23D05B68B9
:106CB000002B20D098471EE06C4BC0180C28C3D87E
:106CC00004F04EF91DC2C2150BC20B0B0B3223C2CE
:106CD0003C00674BC0180728B6D8664B1B68002BD2
:106CE00009D01B68002B06D0200098470AE0A36853
:106CF0001878FFF7C7F8200004F052F9ADE7A06854
:106D0000FFF762F800289FD0F5E7A3681B78002BF7
:106D1000F1D0554B1B68002BEDD01B68002BEAD03F
:106D2000210055489847EDE74F4B1B68002BE2D0F8
:106D30001B68002BDFD021005048F3E7504B1B6845
:106D4000002BD8D05B68002BD5D021004348E9E761
:106D5000FFF7EAF9CFE780884A4B984203D04A4BC5
:106D6000984200D070E7464B1B68002BC3D05B688D
:106D7000002BC0D02100D5E7153B012BBBD963E721
:106D8000FFF798FAB7E7FFF77DFAB4E73F4B1B78B8
:106D9000042B07D100236A4613800179408800F054
:106DA000B5FCA8E7364B1B68002BA4D05B68002B12
:106DB000A1D00100364898479DE7012421420AD01E
:106DC000294B1B68002B04D05B68002B01D00020EE
:106DD0009847012043E78B070AD5264B1B68002BF9
:106DE00004D05B68002B01D020009847022036E7D2
:106DF0000421280008400D4200D131E7254E338898
:106E0000002B21D0013B9BB23380002B1AD1FFF71E
:106E1000DBF800280AD0204B1C70164B1B68002B97
:106E200004D05B68002B01D020009847FFF7C6F81C
:106E3000694601F0F1FC6846FEF7FEFF1D20FEF7F3
:106E400053FF308004200AE7024B187804F030F931
:106E5000F8E7C0462066FF1F9144FF1F0E20000088
:106E600001200000091000001866FF1FFEDFFFFF71
:106E7000AFDFFFFF1C66FF1F0C2000000B2000008F
:106E80000066FF1F0D20000013200000F565FF1FA6
:106E9000FFFF0000F265FF1FF065FF1F10B501F056
:106EA0008BF910BD014B18607047C0461C66FF1F70
:106EB0000B880020162B01D817230420014A1380C9
:106EC0007047C046CA65FF1F00207047074A03008D
:106ED0001188814207D091880020994202D1013067
:106EE0008000101870470020FAE7C0462866FF1F90
:106EF000F0B58F7806000D00C7B01E2F15D1FFF733
:106F0000E5FF051E03D10024200047B0F0BD00229C
:106F10003B003100C078009200F0A2FB0400A81CE6
:106F200000F0C3FBFF23EB70EEE7264B0624039330
:106F30001B78FF2BE8D0182FE6D87B08224A013BAC
:106F4000DB0002929A589446002ADDD0029AD318A8
:106F50005B68002BD8D00878002802D14B78012B31
:106F600002D10624122FCFD107AFAB8869780097E2
:106F70006446AA68A047041EC6D1AB78029A5B0893
:106F8000013BDB00D318390030005B689847041ED2
:106F90000BD1AB78042BB6D0039A310010782200C5
:106FA000009700F05DFB0400AEE76A78002AABD1E1
:106FB000AA7805A93B88087130000A704B80FEF75B
:106FC00047FBA0E79444FF1F40B600111D4B37B5A7
:106FD000050098420BD000290AD1FFF777FF00285F
:106FE00005D11948FFF772FF002800D0058037BD92
:106FF00001291AD1FFF76AFF041EF8D001235B4272
:107000000380A378FF2BF2D0FE2B07D00023E0787B
:107010001422009329001E3300F022FBA01C00F074
:1070200044FB01235B426380E1E70229DFD10139A0
:1070300001F0AEF80028DAD12800FFF747FF041E60
:10704000DFD1D4E7FEFF0000FFFF0000022210B5F1
:10705000074B52421A80074801325A809A80DA80E0
:1070600000F06EFA044801F015F8002010BDC0468B
:107070002866FF1FF16E0011CD6F00110388F7B570
:107080000400002B02D102252800FEBD4268022127
:10709000137825485268FEF7A5FD00282ED0234F0F
:1070A00001253A88002AEFD0802321885B02012540
:1070B0009B1A9942E8DC0C2004F022F8061E31D01D
:1070C0003B8822889C4600231800019561469DB2AA
:1070D000491989B2AA421BD8002801D062443A80DB
:1070E00000233000082208C0210004F0E1F8104A13
:1070F0001368002B13D100251660C5E762680221D2
:1071000013780C485268FEF76DFD0028C7D1BAE726
:1071100060681D014019418101330198D6E71A00CA
:107120001B68E6E71325AFE7AEB600119244FF1FD8
:107130002466FF1FACB60011014B18707047C046A3
:107140009444FF1F14230A0010B51A40194204D0BA
:107150000122102101F038F810BD4B06F9D40120AE
:1071600088434000F8E710B514008B0604D50122CF
:10717000102101F029F810BD08230A001A40194215
:1071800002D14BB2002B0FDA102101F01DF80028BC
:1071900008D02300F9331B78002BECD0F834237887
:1071A000012BE8D10020E6E703208907FAD4E2E7C3
:1071B000F0B51F00184B85B01C6801900291039236
:1071C000002C27D1200005B0F0BDA5683301ED18D3
:1071D0006B89019A934211D3029A93420ED8002FE1
:1071E00004D10A9B002B10D12C00EBE73B0029783F
:1071F000039A6868FEF7F6FC0028F2D10136B6B2B1
:10720000A388B342E1D82468DAE7A3680A9A5B89C5
:107210001380E9E70026F3E72466FF1F37B50C006B
:107220000A8849880123914217D3002A15D0651D89
:1072300023792A0002210A48FEF7D4FC10230028F3
:107240000BD023796188208800242A000094FFF75E
:10725000AFFF0A23A04200D0230018003EBDC04665
:10726000AEB6001113B50A00088849880123884288
:107270000BD8002809D00024137905320094FFF7B9
:1072800097FF0A23A04200D02300180016BD13B5B3
:107290000A0008884988012388420BD8002809D0B1
:1072A0000024137905320094FFF782FF0A23A042DD
:1072B00000D02300180016BDF0B58BB003904A88AB
:1072C00008880E000123824255D3002853D00023A2
:1072D000012704AC23700022718813000092FFF78D
:1072E00067FF051E3ED02078002835D12B78022B71
:1072F00018D167706A8983000130E31880005A80D2
:1073000069680222201803F0D3FF23780133DBB22F
:107310002370042B19D93B006889013080B2002BFF
:10732000D9D01FE002236370122358436A892318BF
:1073300004305A8069681022201803F0B9FF2378BE
:107340000133DBB22370002BE5D10C4A6B899B180B
:107350005A425341DBB2DFE76378012BE4D12B784B
:10736000022BC7D022780A23002A04D021000398D8
:10737000FEF798F9002318000BB0F0BD0100FFFFE5
:107380000F4BF0B504001868002816D083685D899B
:10739000A54207D88288AE18B44203DA12019A18BF
:1073A000934201D10068EFE71E005F891036A742C3
:1073B00004D1002900D00D801800F0BD3300EFE7A4
:1073C0002466FF1F70B505000C0008880021FFF738
:1073D000D7FF03000120002B04D022002800197AD7
:1073E000FFF7C1FE70BDF7B50C000025019023002A
:1073F000F6331B78AB4201D800200AE06B00E65A56
:1074000000213000E718FFF7BBFF002802D12680DB
:107410000130FEBD017A0198FFF794FE002802D0EA
:107420003B882380F5E70135EDB2E0E710B50400B5
:1074300008880021FFF7A4FF03000120002B03D0E0
:107440002000197AFFF77EFE10BD0000054B1B6877
:10745000002B01D1180004E09A6852898242F6D1CB
:10746000988870472466FF1FF0B50E27002687B066
:10747000039302ABFF183E8005001F4B40891400A8
:10748000984207D02B78013000976A6880B2FFF7E6
:107490008FFE060002212B7818486A68FEF7A2FBCF
:1074A00000280FD06C892000FFF7D0FF002802D001
:1074B000013C0419A4B2039B002B00D01C803000B7
:1074C00007B0F0BD02212B780D486A68FEF78AFBF1
:1074D0000028E7D102212B780A486A68FEF782FB70
:1074E000002807D0002EDED03B88A342DBD1748970
:1074F000013CDFE76C89DEE7FFFF0000AEB600115C
:10750000ACB60011AAB6001170B504000D0016004B
:10751000FFF7DCFC002803D083781720FE2B05D072
:10752000002E04D129002000FEF738F970BD012299
:107530001021200000F048FE0028F3D0F6E70000FC
:10754000014B18607047C0463466FF1F37B56B4665
:107550009D1D010004000222280003F071FE2B880B
:10756000B02B0ED12379122B09D12300FF339B7846
:10757000012B06D10121608800F0E0F801E01B2B0F
:10758000F8D037BD10B5054B0421187000F098F8FD
:10759000FFF75CFDFEF780FB10BDC0463866FF1F9D
:1075A0000020F0B50BB20F0087B0834234DA274BCE
:1075B000187803F0DDFC051E2BD00378A02B25D115
:1075C00003AE3100FEF7F4F8041E0BD1B378DB07ED
:1075D00024D51F4B06341B68002B03D0310068886C
:1075E00098470400A868002801D003F059FE002C39
:1075F00008D1184A039B1340174A934206D0B37828
:107600001B2B03D00121688800F098F8280003F0B4
:10761000C7FC80200002784007B0F0BD0F4B1B680C
:10762000002B10D0310068889847041EDAD0737898
:10763000002BD7D1B27801A90A704B800C716888F1
:10764000FEF706F8CEE70624F1E7C0463866FF1FCE
:107650003066FF1F00FFFF00000112003466FF1FAD
:10766000F7B50190822040000D0017001E0003F0C6
:1076700047FE04001320002C12D0B02320002370FA
:10768000089BFC226770658026710830002B08D0AB
:10769000190003F00DFE2100019803F0B1FB00205A
:1076A000FEBD089903F0F4FCF5E710B5041E06D002
:1076B0000078FD2803D803F0E3FCFF23237010BDFE
:1076C0000A1F93B210B504000220032B05D8824094
:1076D0000020024BD1529B189C7010BD5866FF1FB2
:1076E0000B8870B5043B04000D000220032B0BD85F
:1076F0000121200000F04CFD03001420002B03D0DA
:107700002900200000F0DEFB70BD000007B513006B
:10771000034A00920A00012100F02CFC0EBDC04675
:107720004979001107B5019203220092024B0A0029
:10773000122100F049FC0EBDC779001107B56B4658
:1077400001AA11800449D88008780633012802D1A3
:10775000190003F0CDFB07BD3966FF1F0C4B10B5B8
:1077600018700023FF210B4A1380138193819380AB
:10777000094A53801370517293819372D174D382EA
:107780001375517703F044FD00F0FCF910BDC046BD
:107790006866FF1F5866FF1F3A66FF1FF0B58DB081
:1077A0006B46002003910C229B5E834200DBB0E01D
:1077B0005D4B187803F0DCFB051E00D1A4E00378D4
:1077C000902B00D09DE006AF01004688380000F005
:1077D00013FA79680400002900D19CE03B88052B4E
:1077E0006ED13B89032B1CD905AC200000F0A2F818
:1077F0006288172A61D83989131D994231D1796875
:10780000237804310291D90738D5607800F08EF9D9
:10781000071E06D0002303712378012B08D0132BF9
:1078200023D0A868002800D178E003F039FD75E086
:107830006288029909A800F0A6F80290380000F0CA
:107840008BF909AA2378387A01920022310000923C
:10785000029A00F012F9380000F064F9029B002B44
:10786000DFD0300000F080F9DBE70378032BD8D1BC
:107870006288029909A800F0D6F8DEE7122B13D12E
:10788000029909A800F0B5F8021EEAD127498B88B1
:10789000002BC6D0887909A92378019161780091DD
:1078A000310000F0EAF8BCE7002302AA938330001D
:1078B000617809AAFFF72AFFB3E71D4B0993F6E7A2
:1078C000042B02D09A1F012AABD8184A043B9B0014
:1078D000995A0029A5D0D218907831003A0000F0CA
:1078E000AEF800289DD13B88042B03D00121300045
:1078F000FFF724FF012C04D1A868002801D003F071
:10790000CFFC280003F04CFB8020039B0002434087
:1079100018000DB0F0BD012800D182E70121300030
:10792000FFF70CFFEDE7C0466866FF1F5866FF1FB4
:10793000010017000B7803704B784370CB788A787E
:107940001B021343438070470A88030002700A88B1
:10795000120A42700A88012A06D14A8882704A882F
:10796000120AC2700420704702208242FBD14A886A
:1079700004309A704A88120ADA708A881A718A88E2
:10798000120A5A71EFE710B50400012082420CD9A7
:107990004B780A781B0213432380834206D1CB78AD
:1079A0008A781B0213436380002010BD022BFBD199
:1079B000CB788A781B02134363804B790A791B02C8
:1079C0001343A380F0E70B8803700B881B0A4370F6
:1079D0004B8883704B881B0AC3708B8803718B881C
:1079E0001B0A4371CB888371CB881B0AC3710820A3
:1079F000704703000120082A14D14A78087812023F
:107A000002431A80CA788878120202435A804A795F
:107A10000879120202439A80CA79887912020243D5
:107A20000020DA80704710B504000120022A05D139
:107A300000204B780A781B021343238010BDF8B551
:107A4000060010200F00150003F05AFC040001206E
:107A5000002C0ED0A0230C22290023806780201D3B
:107A6000002D07D003F024FC2100300003F0C8F9FA
:107A70000020F8BD03F00CFBF6E7F7B51E00009000
:107A800008AB142017001D78019103F039FC041E87
:107A900012D0A2230370019B47704380099B05719C
:107AA00046710C220830002B07D0190003F000FCAF
:107AB0002100009803F0A4F9F7BD099903F0E8FA52
:107AC000F6E737B5041E0FD04388002B0CD00025F5
:107AD000C1881323007A172201950095FFF7CDFF87
:107AE000FF2365806372257037BD000010B50C4917
:107AF00004004A88002A09D08B89002B05D0002079
:107B0000CB8A0222834201D010BD012213000A2039
:107B1000434300204032C854C81842800472F3E73F
:107B20003A66FF1F0023438003707047094B002112
:107B30001A0010B55C88002C06D01C79844203D151
:107B40000A234B43D01810BD01310A330329F1D168
:107B50000020F8E73A66FF1F10B50400407A03F0F2
:107B60008FFAFF23637210BD7047043010B580B2E6
:107B700003F0B6FB002803D00421494203F0C8F902
:107B800010BD000070B50025104CA0682580A581AF
:107B9000A580A84202D003F083FBA56000250C4C11
:107BA0000C4B606D1D80230058331D70A84202D01D
:107BB00003F076FB656500256068002801D003F0BE
:107BC0006FFB013508340A2DF6D170BD0067FF1F29
:107BD000A466FF1FF466FF1F70B5041E09D1054D92
:107BE0002880A881A880A868002802D003F058FB4C
:107BF000AC6070BD0067FF1FF0B54B8885B0019386
:107C0000002343600A7905000F00022A00D07BE0C0
:107C1000CA88032A17D98B685E7819783602DC780F
:107C2000D8790E4399781B7A24021B020C43034334
:107C300053495BBA0B80331D93421ED1042C04D0F0
:107C4000631F022B0ED9012015E0019A4D4B120142
:107C5000D35A002B06D00198FFF7BEFF4A4A13699A
:107C6000013313610421B8682E812C80494203F04E
:107C70004FF96860002005B0F0BD434D042C06D0DC
:107C8000631F022B0FD9EB680133EB60DBE7019A2E
:107C90003C4B1201D35A002B05D00198FFF79CFFF3
:107CA0002B6901332B61374B30000293019B029A01
:107CB0001B010193002301998C468B5213006344EE
:107CC0009C8003939E81FFF750FF039B041E9860E6
:107CD00016D00421B868494203F01AF9FA88010065
:107CE000043A200003F0E4FA0199029AFB888A5AC8
:107CF000043B9B18029A8B522B6801332B60A2E73E
:107D0000AB690133AB619EE71E4B0293019B1E01E1
:107D1000029BF35A002B2DD002998C19A0680028E1
:107D200028D0012A26D1FA889B189BB27352A189C8
:107D3000994217D39B1AC018B96803F0B9FA029B8D
:107D4000A289F35A934200D07DE700222B81A388B9
:107D50002B80A3686B60029BF2520B4A536801337D
:107D6000536070E7084A9368013393600198FFF706
:107D700033FF68E7044A536901335361F6E7C046AD
:107D80006A66FF1F0067FF1F7066FF1F70B5051E44
:107D900015D10B4C0B4B1880230058331870606DB5
:107DA000002802D003F07CFA656525005035606834
:107DB000002801D003F074FA0834AC42F7D170BD4A
:107DC000A466FF1FF466FF1FF0B51700A12285B05F
:107DD000920001934243394B06001B680C009B182C
:107DE000D933FF331D78FDF751FF0430854204DDA0
:107DF0003000FDF74BFF0430C5B2BD4207D33A0057
:107E000000213000019B03F0E3F805B0F0BD29002C
:107E1000380003F0FDF82300C6B250331E70039300
:107E2000019B29006365380003F0A2FACBB20293EC
:107E3000002B02D0039B01361E7000262300503316
:107E400003931B78B34204D8606D002831D1002021
:107E5000DBE7029A2800002A04D0013B1000B3425D
:107E600000D02800F700E719387003F0C1F87860F7
:107E700000280ED03A78019903F01AFA019A3B785B
:107E80000136D3180E4A0193D369F6B20133D36198
:107E9000D4E7039B18706065A74205D1084A1320F8
:107EA000D36A0133D362B0E7606803F0F9F90834AC
:107EB000F2E703F0F5F900236365C8E73409FF1F13
:107EC0007066FF1FF7B50D0007000421686803F016
:107ED0001FF82B89040003702B891B0A43702B8821
:107EE00083702B881B0AC3702E8902250436F6B2D4
:107EF000FB2E15D81B4B9F4214D10C2003F000FA27
:107F00001135011E0CD0902303708E3B0371043B8E
:107F10004380154B8460C680187802F071FF0025FD
:107F20002800FEBD5C237B43104AD31800935833CE
:107F300001931B78002B0FD1030032003800009909
:107F4000FFF742FF019B05001B78002BE8D13800AA
:107F5000009903F025F9E3E7054A0725536A013341
:107F60005362DDE7FEFF00006866FF1FA466FF1F87
:107F70007066FF1FF0B587B0009017200F00160045
:107F80000193FFF7F2FD1325041E19D00C98031E70
:107F900002D00199201D9847030AE370052302AA25
:107FA000A0700430908127700098667003A99380B8
:107FB0000494FFF787FF051E02D0200003F070F93C
:107FC000280007B0F0BD0000F0B587B01F000CAB73
:107FD0001B780391059301210DAB06001C780492D8
:107FE00000F0D6F81425002821D02000FFF77EFDF0
:107FF0000135041E1BD01149059B0A78037001321C
:10800000D2B2131EC68001D101231A000B70227157
:108010003000049B03990097FFF7ACFF051E09D1C0
:10802000230021000648074A093303F079F82800A5
:1080300007B0F0BD002363802370F8E76C66FF1F74
:10804000C37A001130750000F8B505000E00064C2B
:10805000064F2368002B02D03100280098470434D3
:10806000BC42F6D1F8BDC0461067FF1F2467FF1F52
:108070000123064A5B425380002313715362044A72
:10808000136053609360D360136170472467FF1FD0
:108090001067FF1F0200002310B506499C00085915
:1080A000002801D1625010BD0133052BF6D11320F9
:1080B000F9E7C0461067FF1F034A5388181A434266
:1080C00058414042104070472467FF1FF0B585B00B
:1080D00002930AAB1F780CAB1B88009008000E00BF
:1080E00001920393FFF7E8FF05001120002D1BD13B
:1080F0000E48FFF7E1FF04001520002C14D00622E3
:108100000B99A771E01D03F0D3F8019B3000237198
:10811000029B29006371009B66802370039B65624C
:10812000E381FFF791FF280005B0F0BDFFFF0000DD
:1081300010B5FFF7C1FF04000220002C12D06088A8
:108140000121FFF781FF606A002801D002F030FFB3
:1081500028220021200002F09BFF012300205B4227
:108160006380207110BD000030B5074A074C558868
:10817000010013780020A54204D05B1A59424B41FC
:108180005842104030BDC0462467FF1FFFFF00006B
:10819000084A10B501230C00904208D0FFF78CFF6D
:1081A000031E04D0037923405A1E9341DBB218000A
:1081B00010BDC046FEFF0000024B1879431E9841D7
:1081C000C0B270472467FF1F70B504000D00160091
:1081D000FFF772FF002804D10D4B9C4200D01430F1
:1081E00070BD416A03790520002907D012221A4088
:1081F000102A02D10520002EF2D10F20DB06EFD588
:10820000897E0C20A9428941494249420840E7E75A
:10821000FEFF0000030010B5002800D110BD034888
:10822000034A41889142F9D09847F7E72467FF1F36
:10823000FFFF0000002330B5C45CCD5C6C40D4541B
:108240000133102BF8D130BD0F23002210B5C45CD0
:1082500064002243CA54C25CD209013BF7D210BD6C
:108260000200010010B52032103102F051FF10BDA4
:10827000F0B58BB00390102005931700049102F025
:108280003FFF0090102002F03BFF009B1324019061
:10829000002B05D000280CD11324009802F088FE92
:1082A000019B002B02D0180002F082FE20000BB0D0
:1082B000F0BD102002F024FF0600102002F020FF85
:1082C00013240500002E00D1AEE0002819D01022A2
:1082D000002102F0DDFE32002900039802F018FFB1
:1082E000041E0ED133787F2B51D830000099FFF750
:1082F000ABFF009B1B787F2B53D801990098FFF7A9
:10830000A3FF300002F054FE002D02D0280002F03E
:108310004FFE002CC1D1102002F0F2FE060010200A
:1083200002F0EEFE0290002E7CD0002878D03A00B9
:108330000F3223000125121105D00F333B4015B237
:108340005A4253411BB26A1E1201002B33D0049BC8
:10835000D2B298180099029AFFF76CFF013D1022E3
:108360000021300002F094FEADB2049F2D017D1972
:10837000AF4242D0002C33D0300002F019FE029BF5
:10838000002B00D189E7180002F012FE85E72900D2
:108390003000FFF759FF28002549009AFFF74AFFF0
:1083A000A7E729000098FFF74FFF28002049019A0E
:1083B000FFF740FFA5E70F210F4004998A18D9B2B3
:1083C0008F4208D9D15C06A819540133102BF6D17D
:1083D000029A0199C0E7791A48424141C901F2E77E
:1083E0003900300006AAFFF725FF3200039806A9DE
:1083F00002F08EFE10370400BAE7002CBCD130002A
:10840000029906AAFFF716FF320006A9039802F0A8
:108410007FFE082204003100059802F049FFABE717
:108420001324A9E71324AAE7002800D06EE733E756
:10843000B4B60011F0B58BB00F0016000225009005
:1084400000283FD0002A3DD00B1DDBB2180002935C
:1084500002F056FE1135041E34D0FDF757FD05001D
:108460003A000099201D02F06BFFEBB20393E3701A
:108470002B0CDBB22F0A00936370FFB22B0E23701C
:10848000A7700193FDF73CFD1022010006A802F041
:1084900057FF2100029A04AB06A8FFF7E9FE051E6C
:1084A0000DD1039B08223370009B04A9B370019B7C
:1084B0007770F370301D02F043FFFDF72DFD2000B3
:1084C00002F076FD28000BB0F0BDF0B58FB00D00C6
:1084D000149E039004920593002A03D102242000E5
:1084E0000FB0F0BD002EF9D00398FFF7E5FD14247E
:1084F000071EF4D07278337812021A43B3781B0443
:108500001343F27812061A43036A0192934201D38D
:108510000133E3D1002D03D03B7901249B07DED545
:108520000822002106A802F0B3FD059B13240433A2
:10853000DBB21800029302F0E3FD051ECFD0059ACE
:108540000499043002F0FCFE04223100280002F0FD
:10855000F7FE3900102210310AA802F0F1FE2900BE
:10856000029A06AB0AA8FFF783FE041E0FD1082269
:1085700006A908A802F0E4FE0822311D08A802F0AE
:10858000AFFC012807D101990398FDF7D9FC280019
:1085900002F00EFDA3E70124F9E7000070B51C4CC2
:1085A00005002368181E10D0002D14D11A78002A57
:1085B0000CD1981C083202F07BFE02F0F9FD013567
:1085C000002808D123681D70012070BD0A331800EF
:1085D000082202F06DFE2368002BF5D0122002F075
:1085E0008FFE061E0DD0C123216803704570023135
:1085F0001022023002F05CFE23683100587802F04D
:10860000FFFB206802F0D4FC00232360DCE7C046B7
:108610004C67FF1FF8B504002020FDF765FB0D4EE9
:10862000A700BB590500002B0DD000280BD0D8782F
:10863000FF2809D108492A000C55F359074803338C
:10864000611802F06DFDF8BD290002F0F9FB002869
:10865000F0D1F8E76867FF1F5067FF1F6D980011A2
:1086600070B5064D84006359002B05D0D87802F010
:1086700007FDFF226359DA7070BDC0466867FF1FAF
:1086800070B506008CB00C00150000213022684641
:1086900002F0FEFC31001022684602F051FE1D205F
:1086A00021000322684402F04BFE6846FFF7D8FD24
:1086B0002D21040003222800694402F041FE20001D
:1086C0000CB070BDF0B50700160097B001931CAB5D
:1086D0001D7830221EAB00910AA800211C7802F000
:1086E000D7FC102239000AA802F02AFE102200212D
:1086F00002A802F0CDFC0722310002A802F020FE01
:10870000072202AB9818631E9C41019902F018FEE3
:1087100002AB9C732B005A1E934102AAD373002113
:10872000102206A802F0B4FC06221D9907A802F048
:1087300007FE1A2002ABC01806221F9902F000FEA5
:10874000102200990EA802F0FBFD102202AB0EA928
:1087500008781C78013A6040D2B2087001330131C8
:10876000002AF5D10AA8FFF77BFD102212A9040008
:108770000EA802F09DFD102206AB0EA908781D7808
:10878000013A6840D2B2087001330131002AF5D1B4
:108790000AA8FFF765FD044310222098E4B212A94D
:1087A00002F0CEFD200017B0F0BD70B50E00140031
:1087B0008CB00100102268461D0002F0C1FD31009E
:1087C000082204A802F0BCFD2100082206A802F03D
:1087D000B7FD6846FFF744FD04001022280008A9F1
:1087E00002F0AEFD20000CB070BDF8B506000D0023
:1087F00000243719AC4200D3F8BD02F001FD030A92
:108800003B70631CDBB201379D4203D90234F05444
:10881000E4B2EEE71C00EDE773B506000C0002259C
:10882000002819D0002917D0032101A8FFF7DDFF88
:108830006B469A793F231A40013313436A4630004E
:10884000937101A92200FFF71BFF051E04D103222B
:10885000E01C01A902F02CFD280076BD0378580722
:10886000DA08C00FD20080009B0710439B0F18430B
:10887000C0B2704707230B40C908C9000B430370FF
:108880007047000070B50400FFF7EAFE134DA40026
:108890006359002B21D0186A002801D002F088FB10
:1088A0002B59986E002801D002F082FB2B59D86E0C
:1088B000002801D002F07CFB2B59186F002801D052
:1088C00002F076FB2B59586F002801D002F070FBA4
:1088D000285902F06DFB00232B5170BD6867FF1F04
:1088E0000E4B8000C35870B50C00002B0FD09D6854
:1088F000002D0CD02B78201D0B706B784B70A97C51
:10890000FFF7B8FF2B7E23726B69E36070BD102206
:108910000021200002F0BCFBF8E7C0466867FF1F9B
:10892000014B18607047C0466467FF1F074A030089
:108930008000825810B5002A06D0D088984203D112
:10894000012901D1FFF79EFF10BDC0466867FF1FD8
:10895000F0B5264E95B087000B93BB5905000991E1
:1089600012200A92002B31D0D888FFF7A5FB040013
:108970001420002C2AD0280010A9FFF7B1FFBB5902
:108980001E781D6A002E23D00895FDF7FFFA070018
:108990000020FDF701FB0790A379E61D069310ADBB
:1089A0000CA9089800F0E2FA0EA9280000F0D7FA06
:1089B0000B9B0A990493069B09980293079B0396C5
:1089C000019300970EAB0CAAFFF77CFE15B0F0BD2B
:1089D000FDF7DCFA06903000FDF7DEFAE31DA7791B
:1089E000079310AB06000893DAE7C0466867FF1FDD
:1089F00030B50C4C85002A59030085B00120002AAF
:108A00000ED018006946FFF76BFF2B591A78D888EB
:108A1000054B002A00D1054B6A46072100F0D9FB1F
:108A200005B030BD6867FF1F5F8F00116D8F0011AB
:108A300030B5094C8500295985B01022684625318A
:108A400002F036FC2A591121044BD0886A4600F006
:108A5000C0FB05B030BDC0466867FF1F099000111C
:108A600030B5094C8500295985B01022684635314A
:108A700002F01EFC2A591121044BD0886A4600F0EE
:108A8000A8FB05B030BDC0466867FF1F47900011C6
:108A9000F7B54D4F86001020F4590D0002F030FB61
:108AA000F3592062186A132200286CD0033A290077
:108AB0009C6802F0FDFBF3591A780192002A58D104
:108AC0001E6A227D317B944651400122019F114252
:108AD00001D167461740217D914339432175377B8A
:108AE0004F40BC4660460027800701D44F0817401E
:108AF000012102208F40227D82433A432275377B39
:108B00005740BC4660460027400701D497080F40F5
:108B10000420227DBF0082433A432275627D0027F4
:108B200094466046727B42400A4201D167460F403C
:108B30000121627D8A433A436275777B5740BC4688
:108B400060460027800701D457080F400220627D4D
:108B50007F00824317436775767B00227E4076074D
:108B600001D4BA080A400426617D9200B1430A4349
:108B700062756A78002A08D06278002A05D005223A
:108B80000533DA7700221000FEBD04222979114254
:108B900005D1A17C114202D10533033AF1E7019AD4
:108BA00021782C78002A02D10A0021001400182212
:108BB0000429E8D8042CE6D805206043034A05338D
:108BC0001218525CDDE7C0466867FF1FC4B600118B
:108BD00010B50A001121024B00F0FBFA10BDC0468F
:108BE000A39000110B0030B587B001AD2B806B4610
:108BF00004001100981D082202F05AFB2A000B21E4
:108C00002000024B00F0E5FA07B030BDCB90001118
:108C100010B50A001121024B00F0DBFA10BDC0466E
:108C20001F91001113B50B0011006A4613706B46BB
:108C300004000622581C02F03BFB6A460821200073
:108C4000014B00F0C6FA13BD3F91001110B50A00A8
:108C50001121024B00F0BDFA10BDC0468F910011EA
:108C60007FB505000B4BAA00D4580800002C0FD08C
:108C7000666F237FE28821780396266F0296E66E60
:108C80000196A46E0094FDF719FC2800FFF7FAFD89
:108C90007FBDC0466867FF1F10B51721FFF7E0FFD3
:108CA00010BD000070B50A000D00064B0221040043
:108CB00000F08FFA060029782000FFF7D1FF30007E
:108CC00070BDC0466F90001170B586B000236A4633
:108CD0001370836804001D78681E0A2859D801A9FA
:108CE00002F08EFB060633373B3F43474B4F5300A2
:108CF000180000F042F9062312284BD000281BD19F
:108D00006088FFF7D9F90823002813D04279002A98
:108D100047D1264B1A78072312070BD5244B1A6824
:108D20000723002A06D01668002E03D0290001AAC6
:108D3000B04703006A4613706B461B786088002BAF
:108D40002AD1FFF767FC06B070BD180000F06CF97F
:108D5000D4E7180000F087F9D0E7180000F093F985
:108D6000CCE7180000F0ADF9C8E7180000F0C3F92F
:108D7000C4E7180000F0F6F9C0E7180000F0F6F9B3
:108D8000BCE7180000F013FAB8E7180000F013FA77
:108D9000B4E707236A46137069466088FFF782FFCD
:108DA000D1E70523012AC5D1024BB8E7F565FF1FBE
:108DB0006067FF1F6467FF1FF8B52C4F8600F359EB
:108DC00004000D00002B40D0DA8882423DD15A7851
:108DD000062A33D11A78002A2ED0012099681A6AFF
:108DE000097D014206D0157B054203D007225A7047
:108DF0000120F8BD0220014204D0157B054201D0BC
:108E00000922F4E70420014204D0127B024201D07F
:108E10000B22ECE7164B1B68002BE9D05B68002B9C
:108E2000E6D020009847BB5900215B78122BDFD198
:108E30002000FFF715FFDBE70E4BECE7112A04D10A
:108E4000002900D032252900F2E7002D08D12000AA
:108E5000FFF732F9002803D010230279134303717E
:108E600021002800FDF7A8FAC2E7C0466867FF1F87
:108E70006067FF1F6467FF1F70B50E4E8500AB591A
:108E80000400002B13D01B78002B11D10A4B1B6858
:108E9000002B04D05B68002B01D020009847735949
:108EA0005B78122B03D100212000FFF7D9FE70BDA3
:108EB000024BECE76867FF1F6467FF1F6067FF1FD7
:108EC000094B8000C3581020002B0CD01A6A002ACE
:108ED00009D09B68002B06D0127A1B7E101C9A4288
:108EE00000D9181CC0B270476867FF1F70B5030037
:108EF0000D0014000220002A30D000292ED013705B
:108F00000B78081D53704B789370FFF7A7FCE07047
:108F1000012002212B7A23716B7B034063716A7BF2
:108F20000A401343042263716E7B1640334363711E
:108F30006E7BF608F600334363712B7B0340A3710D
:108F4000287B014000200B43A371297B0A40134377
:108F5000A3712A7BD208D2001343A37170BD10B550
:108F60000A0001000120FFF7C1FF10BD10B50A0083
:108F700001000220FFF7BAFF10BD70B506000C001B
:108F80000220002E30D000292ED07378201D0B70C7
:108F9000B3784B70F178FFF76DFC012235792572BB
:108FA00071794B1008001340934010400343881020
:108FB00010408000C9080343C9000B436373B179B3
:108FC0004B100800134093401040034388100240A8
:108FD0009200C9081343C9000B4321202373FCF7F7
:108FE00083FE854201D2122070BD2220257AFCF733
:108FF0007BFE8542F7D823781820042BF4D86378B9
:10900000012BF1D80020EFE7030010B50220002962
:1090100009D0002B07D00322481C0A7019000D321A
:1090200002F046F9002010BD03000222080010B52E
:10903000002B06D0002904D00E32591C02F038F95A
:109040000022100010BD030010B50220002909D035
:10905000002B07D00422481C0A7019000C3202F0C1
:1090600027F9002010BD10B5FFF7DEFF10BD03008B
:109070000220002906D0002B04D0052200200A700F
:109080001B784B70704703000220002B08D000298A
:1090900006D05B7800200B70013B082B00D91830FC
:1090A0007047030010B50220002909D0002B07D01B
:1090B0000622481C0A7019000A3202F0F9F8002052
:1090C00010BD10B5FFF7B0FF10BD02000B0002206D
:1090D00010B500290ED0002A0CD007211970118874
:1090E00059701188090A997011180822D81C02F0C9
:1090F000DFF8002010BD03000A00022010B5002B8D
:109100000CD000290AD099785878090201431180BF
:10911000901CD91C082202F0CBF8002010BD0300DF
:1091200010B50220002909D0002B07D00822481CC6
:109130000A701900921802F0BBF8002010BD02005E
:109140000B00022010B500290BD0002A09D00921FC
:109150001970117818185970511C062202F0A8F8DD
:10916000002010BD10B5FFF75FFF10BD02000B001F
:10917000022010B5002A09D0002907D051781970B3
:1091800011180622581C02F093F8002010BD0300AD
:1091900010B50220002909D0002B07D00A22481C54
:1091A0000A701900063202F083F8002010BD10B5D5
:1091B000FFF73AFF10BD02000B00022010B5002A95
:1091C00006D0002904D018005178FFF753FB002087
:1091D00010BDF0B585B017001E006A4606230500D5
:1091E000080091819380FEF7C0FC1324011E0290B9
:1091F0000CD03800B047041E05D1280001A9FEF7A5
:109200006FFA041E02D0029802F04AF82800FFF715
:1092100001FA200005B0F0BDF0B504008BB001915B
:1092200015000021102202A801F032FF334EA700E2
:10923000B85900283CD0C388A34239D10378002B09
:1092400036D14278062A18D1020001005532353154
:109250000C3006ABFFF7A9FA002829D12000FFF750
:109260002FFE020006A902A802F022F8200002A99F
:1092700001F00EFE01200BB0F0BD816E002917D069
:109280000B8A112A28D19D420ED101981231093A38
:1092900001F026FE012807D1BB5920009D6EFFF783
:1092A0000FFE29000200DEE732212000FFF7D8FC84
:1092B0002000FEF701FF061E1BD0416A002918D0CE
:1092C0000B8AAB4215D108220198123101F008FE39
:1092D00001280ED1716A0AE09D42E9D10822019865
:1092E000123101F0FDFD0128E2D1BB59996E8A7E51
:1092F000B9E7200002F0ACF8BCE7C0466867FF1F82
:10930000F0B56B4D87007E5985B03378029003939A
:10931000002B00D087E0B368346A01937078062888
:1093200017D101221B7D134202D0217B114218D19B
:109330000222134202D0217B114251D10422134256
:1093400003D0237B134200D08BE0019B5A7DEB5965
:1093500091E007380428F8D802F052F8032E42674B
:109360008300B36E002B03D11C2001F0C9FEB06650
:10937000EB599C6E002C1CD010220021200001F023
:1093800087FE0298FFF79CFD01002000FFF72DFAF1
:1093900001F036FF2082200008211230FFF725FA65
:1093A0000298FFF78DFDA076EB592100D888FFF7D2
:1093B0000FFC0822EB591CE0B36E002B05D01A00FD
:1093C000198AF0881232FFF70DFC0222019B197DE9
:1093D000EB5911423DD0207B10423AD0073208E0D1
:1093E000F488FCF7EBFD01002000FFF711FC0A22D6
:1093F000EB595A70029B9C002A595378073B042B67
:1094000011D8D088FEF758FE00284ED0C3895A08DC
:10941000D2182849029B0298CB542B594118043387
:10942000254801F07DFE05B0F0BDFCF7AFFD03005F
:109430000120834201D100200393EB59DE88FCF721
:10944000ABFD039902003000FFF7ECFB019AEB59EA
:10945000117D042211420CD0217B114209D00B2234
:10946000C7E7F688FCF74CFD01003000FFF7EEFB84
:109470006BE7019A527D01210A4204D0607B0842C9
:1094800001D00C22B5E702210A4204D0607B0842D9
:1094900001D00E22ADE704210A4204D0627B0A42C9
:1094A00001D01022A5E71222A3E7FA225200B0E76A
:1094B0006867FF1F6C67FF1F7798001110B5064B98
:1094C0001A780423100018401A4200D00348FFF70E
:1094D00027FA002010BDC046F565FF1F9844FF1F06
:1094E00070B50400FFF7D4FA051E43D12000FFF742
:1094F0007FFA234EA400A0598268937CDB0708D52D
:109500000321036A1B790B40012B02D1017F0B431E
:109510000377431DD97F8B1E022B0DD8022900D063
:109520000121C088FCF7A0FF042133591A7F59702C
:109530000A431A77280070BD01290CD1022310229A
:10954000437000210C3001F0A3FD3059102135305B
:10955000FFF74BF9EEE70529ECD10223D118437050
:1095600010220C3001F0A4FE04233259117F0B436A
:109570001377EAE708251828DCD1053DDAE7C0466D
:109580006867FF1FF0B58BB0059143887E4F9E0042
:10959000F45915000493002C15D1012902D00020A4
:1095A0000BB0F0BD101D57781678FFF757F9EB6830
:1095B000320002932B7A0499019300903B00200023
:1095C000FCF71CFFEBE7E388049A934201D00820E4
:1095D000E6E72378012B00D1D4E0059B581E09282B
:1095E00000D9CFE001F00CFF05CE0A29CC506C85E4
:1095F0009AB229000498FFF773FFD1E720002900F1
:109600001022453001F054FEB9594B78042B02D199
:10961000013B4B70C3E70B000A00253335320C3198
:109620000498FFF795F90498FFF702FA0522431E04
:109630009841BB59C0005A70B2E72000290010229F
:10964000553001F035FE049B4F4C9D00295904987C
:109650000A0006AB55320C31FFF77AF9295910226E
:10966000453106A801F03CFC012808D10498FFF719
:10967000F7F90590002804D106222B595A70059855
:109680008EE708230593FAE763780C2B7AD1E36E13
:10969000002B03D11C2001F033FDE066BB59D86ECE
:1096A00000286FD01022290001F002FEBB59049857
:1096B000DC6EFFF705FC0D22A076BB595A706EE7F1
:1096C000E06E00285ED063780D2B5BD12B880822DA
:1096D0000382A91C123001F0EBFDBB599A68517D41
:1096E0000222114226D0186A407B104222D00C324E
:1096F000E4E763780E2B45D1236F002B03D11620AE
:1097000001F0FEFC2067BB59186F002803D010221F
:10971000290001F0CDFD0F22BB59CFE763780F2B55
:1097200030D1206F0622691C103001F0C1FDBB59F9
:109730009A68517D0422114203D0196A497B114273
:10974000D5D100210498FFF78BFA28E7636F002B2F
:109750000DD0BB59586F0028F3D01022290001F01A
:10976000A7FD0122BB5952425B6F1A61E9E7142041
:1097700001F0C6FCBB5960675B6F002BE9D126E79F
:109780002978DFE707200BE76867FF1F10B5064C55
:10979000207001F0A5FC06212078FDF791FF034819
:1097A000FEF778FC10BDC0467B67FF1F2D890011B6
:1097B00000200BB270B50D00834216DA264B1878E4
:1097C00001F0D6FB041E0DD00378922B0ED0A02BF7
:1097D00037D0224B1878FF283AD0210001F010FB37
:1097E000002835D180200002684070BD43780E2BE0
:1097F0000BD03E2BEDD18378052B12D0082BE8D16E
:1098000081798088FFF7D8FA08E0154B82889A4260
:10981000DFD183681878591CFEF7C0FE002817D1E5
:10982000D7E7104B1B785B0712D50F4B1B68002B3B
:109830000ED09B68002B0BD0C289811D8088984771
:10984000ECE7FFF741FAA068002801D001F028FDFD
:10985000200001F0A5FBC5E77B67FF1F9144FF1FB8
:1098600018200000F565FF1F6467FF1F10B5007822
:10987000FFF712FA10BD10B50078FFF7FDFA10BD22
:109880000C234343084A10B59B185A68002A03D09A
:10989000012901D1904710BD9B68002BFBD0002906
:1098A000F9D19847F7E7C0469867FF1F10B516280B
:1098B00013D801238340094A946B1C439463506B73
:1098C00098435063D46B20009843012901D12000B4
:1098D0001843D063116B0B43136310BD008000402D
:1098E000F0B500240127154B85B0DA6B144E0392B6
:1098F0001A6C0192DA64019BE3403B4217D0039D4E
:10990000E5403D400295E5B202992800FFF7B8FF17
:10991000316A736A002908D03900002B01D00299FE
:1099200079402800FFF7C2FF01E0002BF9D1013494
:109930000C36172CDFD105B0F0BDC04600800040CA
:109940007C67FF1F10B5012402002000162A08D8EA
:10995000054B5968D140214204D01868D0400123FA
:10996000184010BD186DF9E700800040162807D890
:109970000122064B8240002903D0D9680A43DA60ED
:109980007047D9689143D960FAE7C0460038004073
:1099900030B5162818D8032444430F4BE25C1B193A
:1099A0009C785D7801232D1B0135AB40013BA34022
:1099B000A140DB430C00122807D808499200521836
:1099C000116819402143116030BD054A11680B40F0
:1099D00023431360F8E7C0460BB7001108F00040BE
:1099E00014F00040C21F70B5D4B20623092C0BD866
:1099F0000125084C9540002908D00021FFF7C8FF39
:109A000023682B4323600023180070BD2368AB43F9
:109A1000F8E7C04600380040F0B5162826D8214B9C
:109A20001B185B78022B21D1032444431E4A1F4E8E
:109A3000A35C12199478012215008540B76B013C94
:109A4000E4B23D43A240B563194C122815D89B00DF
:109A500000290CD117495B1899680A439A600123C1
:109A6000205C154A834011680B431360F0BD114917
:109A70005B18996891439960F1E70E4B00290DD16D
:109A800059690A435A61225C1328E8D00123203A1D
:109A900093400A49086803430B60E7E7596991431B
:109AA0005961F0E77C67FF1F0BB700110080004091
:109AB00050B7001100F00040A0F00040A4F00040BA
:109AC000F8B500241B4E1C4D1C4B1B5D012B1FD1F8
:109AD000184A9269E2401A420BD00122AA569340DA
:109AE0002200143AD2B2022A09D815494A6913430E
:109AF0004B6101340C360235172CE5D1F8BD00223C
:109B0000AA560F499200521891680B439360F0E7F0
:109B1000022BEED1E7B23800FFF714FF01235840C3
:109B2000C1B23800FFF778FF3800FFF70BFF7077FE
:109B3000DFE7C0467C67FF1FDDB600117D67FF1FB2
:109B400000F00040012202388240054B002903D07A
:109B500059690A435A617047596991435961FAE753
:109B60000038004070B504000D000520162C1AD8EE
:109B700000212000FFF7FAFEA31E012B03D80121CC
:109B80002000FFF7DFFF00212000FFF72BFF01225D
:109B90000A49A2400A4B4868012D05D102431B190E
:109BA0004A605D70002070BD9043486002211C191E
:109BB0006170996991439961F4E7C0460080004063
:109BC0007C67FF1F10B516280AD80122074B824078
:109BD000002906D019680A431A600121FFF7C2FF65
:109BE00010BD196891431960F7E7C0460080004036
:109BF00070B505000520162D17D80C2300246B43E3
:109C00000A4A21009B181C70094B28005B195C70E4
:109C1000FFF7A8FF0123AB40200006490A681A435A
:109C20000A6005490A689A430A6070BD9867FF1F79
:109C30007C67FF1F348000403080004070B5040016
:109C40000E00FF2813D003250540FFF7D1FF084A77
:109C5000A3089B009B183F22ED00AA40AE40196864
:109C600020009143314319600121FFF77FFE70BD51
:109C700018380040F8B505000520162D25D80C240D
:109C80006C43124BE4186368002B03D1A3680D30BA
:109C9000002B1AD0022201270D4B00215B195A70AC
:109CA00028002770FFF75EFF63681E1E08D0A368B8
:109CB0003E00002B04D02800FFF744FE4640F6B2D9
:109CC00028003100FFF7F2FD0020F8BD9867FF1F64
:109CD0007C67FF1FF7B5C420FF222B4B800019586B
:109CE000002491437F3A0A431A508022274F5202A0
:109CF000274E1A60274B1D5D002D21D0A31E012B7E
:109D000003D80121E0B2FFF71DFF012D18D11F4B31
:109D10009B69E3402B4213D0E3B218000193FFF795
:109D200011FE01000198FFF74DFFE3B2143B022B37
:109D30001DD801217156184A8D405369AB435361B8
:109D40003B7F002B0DD0E5B22800FFF793FF2800E2
:109D5000FFF7F8FD7B7F0100834202D02800FFF768
:109D60008FFD01340C370236172CC3D1F7BD01210A
:109D700000237156F3568D40074A9B009B189A6842
:109D8000AA439A60DCE7C04600E100E07C67FF1F61
:109D9000DDB600117D67FF1F00F0004010B5040024
:109DA0000520162C0CD801212000FFF7DBFE012333
:109DB000044A002011194B70A34091690B43936131
:109DC00010BDC0467C67FF1F70B50E001500040073
:109DD000FFF70EFF0C236343094A20009B189D6088
:109DE0005E60FFF747FFF021064B074A8900051E1A
:109DF0005A5002D02000FFF7FBFE280070BDC0467D
:109E00009867FF1F0000FF1FE198001170B5134D08
:109E100007202C78002C1FD1982221005200280006
:109E200001F0D6F90123C420FF222B700C4B8000D7
:109E30001C635C630B4B1C605C600B4B19589143BB
:109E40007F3A0A431A50802252021A600D20074AB4
:109E5000074901F025F9200070BDC0467C67FF1F4F
:109E600000800040A0F0004000E100E0D59C00111F
:109E7000C19A0011030010B50620072B09D8054A26
:109E8000137000F0FDFFD7210020034B034A890027
:109E90005A5010BDC044FF1F0000FF1F151BFF1FBD
:109EA00070B51D0002240C2910D8094ACA40D207F7
:109EB0000CD5FBF725FF041E08D1059A049928004C
:109EC000FBF73AFFFCF7A8FDFFF7F8FA200070BD9A
:109ED0001210000030B50D7802232C009C4318426C
:109EE00001D02B431C0008252300AB43284201D09E
:109EF0002B00234320241D00A543204201D01C43F6
:109F000025002A230D70184204D011781E3B0B4304
:109F1000137030BD0028FCD10C2113788B43F7E778
:109F2000F8B51D0006AB1B88140007AA0E000B2015
:109F30001778002B27D10A78022A49D14A6850782D
:109F400011780002244A08438018042840D801F000
:109F500057FA03121D1B2300F06801F011FA021CCE
:109F6000C0B2B84200D93A1CD2B22000F1682A80AF
:109F700001F09EF906E00222F3681B882A80237014
:109F80001B0A63700020F8BD0622EEE701232B8038
:109F9000F3681B782370F5E7F368002B16D00822CE
:109FA0002A801A8822701A88120A62705A88A2704F
:109FB0005A88120AE2709A8822719A88120A62718B
:109FC000DA88A271DB881B0AE371DBE72B80D9E713
:109FD00001202B80D7E7C04600D6FFFFF7B516005B
:109FE0000A781D0008AB1F880C000123022A18D133
:109FF0004A685078117800022B4A084380180328D9
:10A000000FD801F0FDF902254439E06801F0B8F9F4
:10A01000C0B20723B84204D37B190193152B02DD8C
:10A020000D231800FEBDE0682A003100C01901F0C0
:10A030003FF96B4600209B88E268D0541B4B1B689D
:10A04000834203D01B68834200D098470023E8E78F
:10A050000B23002FE5D1022DE2D1737832781B0259
:10A060001343E2681380114B1B68002BEED01B6872
:10A07000002BEBD00120E8E70B23002FD1D1062DD8
:10A08000CED12A003100E06801F012F9DEE70B239F
:10A09000002FC6D1012DC3D132787533012AC0D823
:10A0A000E3681A70D2E7C04600D6FFFF8869FF1F39
:10A0B00070B50C001500072837D801F0A1F9041479
:10A0C00036361B36242E182015290BD8184E16228A
:10A0D0000021300000F0DCFF22002900300001F0F8
:10A0E000E7F8002070BD18200229FBD11288114B1F
:10A0F0001A80F6E718200829F4D10A000E48290032
:10A1000001F09EF8EDE718200129EBD10B4B1078F8
:10A110000B49DA69FFF7DEFEE3E718200129E1D1F8
:10A12000064B10780749DA6BF4E70220DAE7C046FD
:10A130007069FF1F3E45FF1F3445FF1FC444FF1FCA
:10A14000EC44FF1F0C45FF1F030010B50020DB0788
:10A1500004D50721024A034800F08CF810BDC04620
:10A1600068B70011C444FF1F054A030010680028A7
:10A1700003D082889A4201D1806870470068F6E770
:10A180008C6BFF1F0A88030008009A4204D08A885B
:10A1900004309A4200D0002070470000F8B5F82241
:10A1A00000230D4F0D4E79680500424333709942EC
:10A1B00000D07B600A4C0021200000F069FF0023E2
:10A1C0001A007C60AB4202D100203370F8BD01332D
:10A1D0002280DBB2F834F5E78C6CFF1F886CFF1F20
:10A1E000906BFF1F73B56B46019006006846150023
:10A1F0001980FCF743FF041E11D1002D0FD0768982
:10A20000002E11D00C2000F07BFF00280ED0084A51
:10A210000460136886808560002B02D110602000E6
:10A2200076BD1A001B68F7E70224F8E71324F6E767
:10A230008C6BFF1F012100220A4B10B549420A4CCA
:10A24000198099809A719A70084B207001201980AA
:10A250005A60FFF7A3FF2078FCF76EFF0448FDF774
:10A2600019FF10BD9069FF1F946CFF1F8C6CFF1FBE
:10A2700021A30011022310B5002802D0FFF7B2FF7E
:10A280000300180010BD0000030010B50020DB071C
:10A2900004D50421024A0348FFF7A4FF10BDC046BD
:10A2A0007CB700114445FF1FF0B50E2687B003931D
:10A2B0000CAB1F8802ABF6180500080031000292B3
:10A2C000FDF75EF804000120002C0FD03088FFF766
:10A2D0004BFF03000E20002B08D05E68002E05D037
:10A2E00021002800039B029A0097B04707B0F0BDF9
:10A2F0000A4B10B5984207D10122002352420A802E
:10A300008B708A808B7110BDFFF73CFF0028FAD05C
:10A3100001235B42038000238370F4E7FFFF00000A
:10A32000F8B5050001290AD1134E00243388F82717
:10A33000AB4219D028001149FFF7DAFF06E00229E5
:10A3400004D10139FDF724FF0028EDD0F8BD3B0012
:10A3500063437268D018D35A002B09D03A00002109
:10A3600000F096FE0134E4B2054B1B78A342EED810
:10A3700001235B423380DDE78C6CFF1F9069FF1F78
:10A38000886CFF1F10B5FFF7FDFE0300002083421D
:10A3900000D0987810BD0000F0B589B01C000EAB5D
:10A3A00080CB03901E8810AB1B78049202930B7A2B
:10A3B0000D00DB0616D42B780593022B24D00498CD
:10A3C000FFF7D2FE002812D003689C46002B0ED067
:10A3D000029B2200019329003B00644603980096EB
:10A3E000A04705E00498FFF7BFFE002802D10E2029
:10A3F00009B0F0BD8368002BF9D00A222900039828
:10A4000098470028D7D0F3E76B6858781A786B4BD9
:10A41000000210439842D2D8043B984210D2684BB5
:10A42000984242D015D8674BC0180128C7D80B20D6
:10A43000002EDDD1EB681A7859683A80200028E0B8
:10A44000614BC018032800D979E000F0D9FF846A75
:10A45000789E5E4B9842B2D10B20002EC8D10123CA
:10A460003B80EB6831001B7823706889013080B233
:10A47000FCF786FF3A88031E0ED0017802328A1854
:10A480003A80428962704289120AA2705968027841
:10A49000E01C00F00DFF06E004323A803100042297
:10A4A000601C00F0F5FD0020A2E70B20002E9FD1DC
:10A4B000EB6807A91E8804233B80330A300026700E
:10A4C0006370FCF75DFF051E28D004AB9A890E234C
:10A4D00004A95B183E49C668FCF7C6FF00280BD1EB
:10A4E0002B783C486A680599FBF77CFB002803D170
:10A4F000012304AA5B42D3813278022A06D1716813
:10A50000201D00F0D5FE3B8802333B800E2304AAB9
:10A510009B181B88A3701B0AE370C4E704ABDE81A1
:10A52000F4E70B20002E00D062E7E9680398FFF7FC
:10A5300029FF02233B802070000A6070B3E70B20E4
:10A54000002E00D054E70222EB681B883A8023706B
:10A550001B0A6370A7E7E86800F012FFC2B20300AD
:10A560000720B24200D243E70DD00299DBB2711846
:10A57000994202DB921BD3B20293029BE9681A0054
:10A580003B8089195AE70023F6E70B20002E00D004
:10A590002EE70722EB683A801A7822705A786270A8
:10A5A0005A88A2705A88120AE2701A792271DA88DF
:10A5B0006271DB881B0AA37175E7C046042900009D
:10A5C0000228000000D8FFFFFFD6FFFF032800008D
:10A5D000FFFF0000ACB60011F0B58DB06B46002057
:10A5E000089120229B5E83423DDAA64B187800F04A
:10A5F000BFFC071E32D00378B02B2CD10079023873
:10A6000016281FD800F0ACFD17001E001E001E000B
:10A6100031001E0096001E001D011E0052011E008A
:10A6200073011E00CD011E0050021E001E001E0000
:10A630008E021E00E302944B94491B8878880B809D
:10A64000FBF710F83800FCF781FF914B1B68002BDB
:10A6500001D038009847380000F0A2FC8020089B09
:10A660000002434018000DB0F0BDF62200218748DB
:10A6700000F00EFD0BAA3B7B7989388900923A00E5
:10A680000D32FCF795FD0400804B1B78002C3FD168
:10A6900046E0804B788805937F4B4100CB5A0BAE48
:10A6A000073BDBB232880293002301937B4B2100EE
:10A6B00006930093059BFFF76FFE744D002810D1A1
:10A6C000069B3A8A1B889A420BD1380005991230B2
:10A6D00000F006FC002804D02B7862899B00EB1860
:10A6E0005A80162306A81B18328820007989FCF7A7
:10A6F000BBFE2B7804009A00AA1851880029C3D009
:10A700000133DBB22B70002807D006A9C98A9180DB
:10A71000634A12889A42BCD802E0012149429180E2
:10A72000002B04D059497888FAF7D0FF8AE73E8990
:10A730000A2479E000253E89574B06937B88069AC8
:10A740005B009B5A033B9D4202DB002DF0D05BE097
:10A75000162206A812183B7B798900923A00300035
:10A760000D32FCF725FD0590002858D04689017A66
:10A770007888FCF7E7FC041E44D1464B78880793A1
:10A78000069B4100C95A454B0439C9B206AAD28A70
:10A7900006930291019400930599079BFFF7FCFD36
:10A7A000041E2FD1069B39491A88931C002D26D1EF
:10A7B0004B807988384B4900CB5A5119033B8B4267
:10A7C00020DD059B31485B8941190B71A91C0135BE
:10A7D000C9B2EDB2059145191B0A2B71059B2D4994
:10A7E0000433181800F064FD2C4B059A1B88D3180D
:10A7F000DDB22C4B9E4205D00136B6B29CE74988AB
:10A800009942D6D0002D0CD0204C2800618800F051
:10A81000BFFB207021007888FAF768FF12E7059CDB
:10A82000F0E7002C00D183E77B78142B00D109E7F7
:10A8300016493B794E800B700C717888FAF708FF47
:10A8400000E7162406ABE41821003889FCF798FDD0
:10A85000011E00D1B7E1788822880F4C45002C5B9F
:10A860000A4D013CE4B2029400240F4B0194009580
:10A87000FFF792FD041E00D014E129007888FAF752
:10A8800045FFDFE6946CFF1F3044FF1F9869FF1FF0
:10A890008C69FF1F926AFF1FC865FF1F886BFF1F2F
:10A8A0002E44FF1FFFFF00009A69FF1F162406AB0E
:10A8B000E41821003889FCF763FD011E00D182E114
:10A8C00078882288AE4C45002C5BAE4D013CE4B24A
:10A8D00002947C89AC4B01940095FFF75DFD041E4A
:10A8E00000D0DFE029007888FAF71AFFAAE60025F1
:10A8F000A44B1D803B00FE331B78A24A7888079248
:10A90000AB4208D99E4B12880693069943005B5AC6
:10A91000013B9A4203DB0799FAF70CFF92E61624F3
:10A920006B00FB18059306ABE418059B2100188902
:10A93000FCF726FD011E03D1059B01241E8973E748
:10A940007888924B2288069C099343001B5B904EAB
:10A95000013BDBB20293002300960193099BFFF7B2
:10A960001BFD041E02D0059B1E895DE77B88069AAD
:10A970005B009B5A079A108832881218934202DCB7
:10A980001B1A013B33807F4C023032880999001931
:10A9900000F08EFC2388328801359B182380EDB2AD
:10A9A000A8E70BAA3B7B7989388900923A000D32DF
:10A9B000FCF7FEFB00250590059B002B04D10A2423
:10A9C000002D00D16EE060E0059B7888197AFCF7D5
:10A9D000B9FB0100041E63D1694C6C4B7888069466
:10A9E0000993069B4400E45A694B063CE4B20BAE63
:10A9F000328807930294019100930599099BFFF710
:10AA0000CBFC041E4CD1079B5E491B881A1D002DF0
:10AA100030D14A80059B5B4C5A8963191A716B1CB3
:10AA20009BB2E318120A1A71162306A832881B1863
:10AA300079890598FCF718FDFF21AA1C2E1D033506
:10AA40000B00059092B2B6B2ADB2002803D006ABAF
:10AA5000DB8AD9B21B0AA218651911712B714C4DF2
:10AA6000301D2A884949201800F022FC2B88F6184E
:10AA7000B5B2A1E74988914207D17A880699520078
:10AA8000525AEB18053A9A42C4DC3E4C28006188C1
:10AA900000F0BEFA207021007888FAF755FED1E563
:10AAA000002DF2D13E89BFE6162606ABF61831001E
:10AAB0003889FCF765FC3D000400FF3500282DD0E7
:10AAC000037A9B060CD400227B893989788800920E
:10AAD0003A000C32FFF7E8FB041E10D03E8915E067
:10AAE0003088FFF741FB00281AD08368002B17D06D
:10AAF0002100122278889847041EE4D0EEE7AB7854
:10AB0000002B02D17888FAF72FFE0026AB78002BB5
:10AB100000D097E5002C00D194E585E60124DDE71F
:10AB20000E24DBE7162506ABED1829003889FCF763
:10AB300027FC041E47D0037A9B0611D4154A7B8854
:10AB40001188994203D01448814207D11380134BD6
:10AB5000F8261D780023D9B2A94221D30924A1E700
:10AB60002888FFF701FB00282FD08368002B2CD00A
:10AB70002100122278889847041EDFD092E7C04651
:10AB8000C865FF1F9869FF1F9A69FF1F926AFF1F20
:10AB9000886BFF1F8C6CFF1FFFFF0000886CFF1F7E
:10ABA00031005943546801336018615A0029D2D1E9
:10ABB0003C0008342100F82200F07AFB210078885C
:10ABC000FAF7DAFD3EE501246CE70E246AE71D4B37
:10ABD0001A887B889A4231D07888FAF7D7FD31E518
:10ABE000F823059851684343CD18C95A00291FD04E
:10ABF0003B7A012B0BD16C88AB887888AA1D009416
:10AC0000FFF752FB041E02D000233B722E88F8226D
:10AC10000021280000F03CFA00232B80059B013323
:10AC2000DBB20593084B05991B78064A8B42D7D8AF
:10AC300001235B421380002CCED0F5E500263400C2
:10AC40000596EFE78C6CFF1F886CFF1F70B5040042
:10AC50000E001500FFF796FA031E08D131000548D3
:10AC6000FFF790FA03001120002B02D01C80002077
:10AC70009D7070BDFFFF0000F8B50B4F06003B78DC
:10AC80000D001400FF2B0ED00A2000F039FB011E2E
:10AC900009D0B1230380002346800371C58004815D
:10ACA000387800F0ADF8F8BD8545FF1FF7B50F0007
:10ACB00008A90600088809A90B240988002821D1C1
:10ACC0000234022B1ED1557813782D021D432B0020
:10ACD0008B4301937334002B14D1FB6830001900AF
:10ACE0000093FFF74FFB019C85420BD02A003000F8
:10ACF0000099FFF7ABFF041E04D12A0030007989C8
:10AD0000FFF7BAFF2000FEBDF0B50E7885B00390C6
:10AD10000AA805880120022E0DD14C682778647896
:10AD200024023C43054FBC4205D10398DBB2019697
:10AD30000095FFF7BBFF05B0F0BDC046022900003B
:10AD400010B504000C4800F00BFB0C48A16B00F0A0
:10AD500007FB0B48E16B00F003FB0A48216C00F095
:10AD6000FFFA094B0948196800F0FAFA084B1B680A
:10AD7000002B00D09847FEE77EB5001194B5001176
:10AD8000A3B50011B2B5001104ED00E0C1B500118A
:10AD9000986CFF1F002307B501A80193FFF7D0FFB0
:10ADA000044A0548002110B5121A00F071F9F8F7AD
:10ADB000C5FDFEE79C6CFF1F8845FF1F00000000DB
:10ADC00001B40248844601BC604700BF5522000020
:10ADD00001B40248844601BC604700BF85520100AF
:10ADE00001B40248844601BC604700BF75A9000059
:10ADF00001B40248844601BC604700BF6939FF1FA7
:10AE000001B40248844601BC604700BF594F0100AD
:10AE100001B40248844601BC604700BF8132FF1F75
:10AE200001B40248844601BC604700BF6DBC00000D
:10AE300001B40248844601BC604700BF4550000091
:10AE400001B40248844601BC604700BF514701007D
:10AE500001B40248844601BC604700BF8B52010028
:10AE600001B40248844601BC604700BF5D17000082
:10AE700001B40248844601BC604700BFC51D000004
:10AE800001B40248844601BC604700BF151BFF1F88
:10AE900001B40248844601BC604700BF311B00007A
:10AEA00001B40248844601BC604700BF5125000040
:10AEB00001B40248844601BC604700BFB54C0100A4
:10AEC00001B40248844601BC604700BFA139FF1F9E
:10AED00001B40248844601BC604700BFEDA50000F4
:10AEE00001B40248844601BC604700BFCD4C01005C
:10AEF00001B40248844601BC604700BFE11700006E
:10AF000001B40248844601BC604700BFED4A01001D
:10AF100001B40248844601BC604700BF55490100A6
:10AF200001B40248844601BC604700BFA134FF1F42
:10AF300001B40248844601BC604700BF093BFF1FC3
:10AF400001B40248844601BC604700BFF94C0100CF
:10AF500001B40248844601BC604700BFD1A500008F
:10AF600001B40248844601BC604700BF453CFF1F56
:10AF700001B40248844601BC604700BFF54E0100A1
:10AF800001B40248844601BC604700BF291C000090
:10AF900001B40248844601BC604700BF350E000082
:10AFA00001B40248844601BC604700BF434D010024
:10AFB00001B40248844601BC604700BF014C010057
:10AFC00001B40248844601BC604700BF1537FF1F2B
:10AFD00001B40248844601BC604700BF5118FF1FFE
:10AFE00001B40248844601BC604700BF35550000EB
:10AFF00001B40248844601BC604700BF017F0000E5
:10B0000001B40248844601BC604700BFDD30FF1F29
:10B0100001B40248844601BC604700BF090E00002D
:10B0200001B40248844601BC604700BFC53F000030
:10B0300001B40248844601BC604700BF018900009A
:10B0400001B40248844601BC604700BF851F000070
:10B0500001B40248844601BC604700BF8D3AFF1F1F
:10B0600001B40248844601BC604700BFC56D0100C1
:10B0700001B40248844601BC604700BF3D1800008F
:10B0800001B40248844601BC604700BF114701007B
:10B0900001B40248844601BC604700BF154D010061
:10B0A00001B40248844601BC604700BF0933FF1F5A
:10B0B00001B40248844601BC604700BFB35201009E
:10B0C00001B40248844601BC604700BFC95C01006E
:10B0D00001B40248844601BC604700BFADAE000029
:10B0E00001B40248844601BC604700BFC926000085
:10B0F00001B40248844601BC604700BF691F0000DC
:10B1000001B40248844601BC604700BF3D4B0100CA
:10B1100001B40248844601BC604700BFE548000016
:10B1200001B40248844601BC604700BFA946010043
:10B1300001B40248844601BC604700BF0D520100C3
:10B1400001B40248844601BC604700BF6932FF1F5A
:10B1500001B40248844601BC604700BF657101002C
:10B1600001B40248844601BC604700BF6D3CFF1F2C
:10B1700001B40248844601BC604700BF9938FF1FF4
:10B1800001B40248844601BC604700BF214601006B
:10B1900001B40248844601BC604700BF0134FF1F70
:10B1A00001B40248844601BC604700BF7D18FF1F00
:10B1B00001B40248844601BC604700BFD91B0000AF
:10B1C00001B40248844601BC604700BF9DA900004D
:10B1D00001B40248844601BC604700BFB70E0000BE
:10B1E00001B40248844601BC604700BF1D4B01000A
:10B1F00001B40248844601BC604700BF5539FF1FB7
:10B2000001B40248844601BC604700BF29510100D7
:10B2100001B40248844601BC604700BF79180000B1
:10B2200001B40248844601BC604700BFA54F01003D
:10B2300001B40248844601BC604700BFC94A01000E
:10B2400001B40248844601BC604700BF810E000083
:10B2500001B40248844601BC604700BFB14E000003
:10B2600001B40248844601BC604700BFF136FF1FAD
:10B2700001B40248844601BC604700BFE139FF1FAA
:10B2800001B40248844601BC604700BFE537FF1F98
:10B2900001B40248844601BC604700BF8D12000023
:10B2A00001B40248844601BC604700BFD94901008F
:10B2B00001B40248844601BC604700BFE94C01006C
:10B2C00001B40248844601BC604700BFC5210000AC
:10B2D00001B40248844601BC604700BF59520100D6
:10B2E00001B40248844601BC604700BFE928000061
:10B2F00001B40248844601BC604700BF056A0000F3
:10B3000001B40248844601BC604700BF1D4D0100E6
:10B3100001B40248844601BC604700BF25260000F6
:10B3200001B40248844601BC604700BF456B010080
:10B3300001B40248844601BC604700BFC9A90000AF
:10B3400001B40248844601BC604700BF455101007A
:10B3500001B40248844601BC604700BF213AFF1F88
:10B3600001B40248844601BC604700BFE53A0100D1
:10B3700001B40248844601BC604700BF090E0000CA
:10B3800001B40248844601BC604700BFDD520100A1
:10B3900001B40248844601BC604700BF4134FF1F2E
:10B3A00001B40248844601BC604700BF212400006C
:10B3B00001B40248844601BC604700BF9135FF1FBD
:10B3C00001B40248844601BC604700BF4D1F000025
:10B3D00001B40248844601BC604700BFF30E000080
:10B3E00001B40248844601BC604700BF012400004C
:10B3F00001B40248844601BC604700BF1D3BFF1FEB
:10B4000001B40248844601BC604700BF593CFF1F9D
:10B4100001B40248844601BC604700BF493BFF1F9E
:10B4200001B40248844601BC604700BF055E0000CD
:10B4300001B40248844601BC604700BF9130FF1F41
:10B4400001B40248844601BC604700BFC132FF1FFF
:10B4500001B40248844601BC604700BF091B0000DC
:10B4600000030103020303030402050206020700AE
:10B47000080309030A030B030C000D000E030F035E
:10B48000100311001303140315031603F53C0011F8
:10B49000293D00110000000002000000A2B40011CC
:10B4A000192A0F180A000000F1590000FD240000BD
:10B4B000414601009D770011B1970011256C0011E4
:10B4C000A1750011BD4D0011D9A500118D4A0011C3
:10B4D000ED3E00111D400011000000001616000096
:10B4E00002000000ECB40011F4FFF3FFD2FC0000F6
:10B4F000D94000110000000000000000547579617F
:10B500000056302E3600303030310067697468756F
:10B51000622E636F6D2F7076767800544842320049
:10B520000200000034B50011292A282A272A262AD9
:10B53000252A242A0A18000006640000204E000074
:10B5400000000000000000001F501D000206B400B3
:10B550000001130006000000830200003031323386
:10B56000343536373839414243444546005048590E
:10B570002B36325858504C555330353034005B48D8
:10B58000617264206661756C742068616E646C65BC
:10B59000725D0A004C522020203D20307825303842
:10B5A000780A0050432020203D203078253038781C
:10B5B0000A0050535220203D203078253038780A38
:10B5C0000049435352203D203078253038780A0016
:10B5D000CD510011215200110000000002000000B6
:10B5E000E8B500116F2A6E2A1A18000001A00000A9
:10B5F000000000006410B71DC8206E3BAC30D92697
:10B600009041DC76F4516B6B5861B24D3C71055042
:10B610002083B8ED44930FF0E8A3D6D68CB361CB6A
:10B62000B0C2649BD4D2D38678E20AA01CF2BDBD1E
:10B63000FB349B5F800000800010000000000000D1
:10B6400027580011B16E00114B580011B97200114A
:10B65000CF5800118F720011455900116572001109
:10B66000975900112D740011FF5900112D7400110C
:10B67000315A0011E7730011455900111D72001174
:10B68000BD590011C573001100000000000000004A
:10B69000A35A0011C5730011055B0011C96E00119A
:10B6A000052A042A012A002A022903280128002841
:10B6B0000118001800000000000000000000000059
:10B6C00000000087010102010201010201020303DF
:10B6D00004010301010101010303020103000D0044
:10B6E0000E001000110013001401070108010A01E7
:10B6F0000B011C011D0204020502070208021902C7
:10B700001A021C021D0301030203170002010005B7
:10B7100004000807000B0A001716001D1C01020197
:10B72000010504010E0D011110011413011716017A
:10B730001A19020201020B0A020E0D021110021464
:10B7400013021716030504030807030B0A030E0D63
:10B750000001020307090A0B0E0F1011121417182B
:10B76000191A1B1F20212200219F0011DD9F0011AB
:10B770000000000002000000B2B60011000000004E
:10B7800009AD00110000000002000000B0B6001179
:020000041FFFDC
:1000000000000000513E0011A8B40011A4B400117A
:100010009462FF1F000000000000000000000000CC
:1000200000000000000000000000000000000000D0
:1000300000000000000000000000000000000000C0
:1000400000000000000000000000000000000000B0
:1000500000000000000000000000000000000000A0
:100060000000000000000000000000000000000090
:100070000000000000000000000000000000000080
:100080000000000000000000000000000000000070
:100090000000000000000000000000000000000060
:1000A0000000000000000000000000000000000050
:1000B0000000000000000000000000000000000040
:1000C0000000000000000000000000000000000030
:1000D0000000000000000000000000000000000020
:1000E0000000000000000000000000000000000010
:1000F0000000000000000000000000000000000000
:1001000000000000000000000000000000000000EF
:1001100000000000000000000000000000000000DF
:1001200000000000000000000000000000000000CF
:1001300000000000000000000000000000000000BF
:1001400000000000000000000000000000000000AF
:10015000000000000000000000000000000000009F
:10016000000000000000000000000000000000008F
:10017000000000000000000000000000000000007F
:10018000000000000000000000000000000000006F
:100190006534FF1F5533FF1FC166010000000000DA
:1001A000000000000000000000000000000000004F
:1001B000000000000000000000000000000000003F
:1001C000000000000000000000000000000000002F
:1001D000000000000000000000000000000000001F
:1001E000000000000000000000000000000000000F
:1001F00000000000000000000000000000000000FF
:1002000000000000000000000000000000000000EE
:1002100000000000000000000000000000000000DE
:1002200000000000000000000000000000000000CE
:1002300000000000000000000000000000000000BE
:1002400000000000000000000000000000000000AE
:10025000000000000000000000000000000000009E
:10026000000000000000000000000000000000008E
:10027000000000000000000000000000000000007E
:10028000000000000000000000000000000000006E
:10029000000000000000000000000000000000005E
:1002A000000000000000000000000000000000004E
:1002B000000000000000000000000000000000003E
:1002C000000000000000000000000000000000002E
:1002D000000000000000000000000000000000001E
:1002E000000000000000000000000000000000000E
:1002F00000000000000000000000000000000000FE
:1003000000000000000000000000000000000000ED
:1003100000000000000000000000000000000000DD
:1003200000000000000000000000000000000000CD
:1003300000000000000000000000000000000000BD
:1003400000000000000000000000000000000000AD
:10035000000000000000000000000000000000009D
:10036000000000000000000000000000000000008D
:1003700095AD00110000000000000000000000002A
:10038000000000000000000000000000000000006D
:10039000000000000000000000000000000000005D
:1003A000000000000000000000000000951AFF1F80
:1003B000000000000000000000000000000000003D
:1003C000000000000000000000000000000000002D
:1003D000000000000000000000000000000000001D
:1003E000000000000000000000000000000000000D
:1003F00000000000000000000000000000000000FD
:08183800A070FF1F4118FF1F03
:10184000024981F3088802F05BFB0000A070FF1FD3
:1018500010B502F075FB072804D0122808D0022822
:1018600008D010BD044A0420136B01331363F8E75A
:101870000220F6E71420F4E77066FF1FF8B50700B2
:101880000C0026002500503630785135002804D150
:101890000300287058342370F8BD2978CA00481E08
:1018A0008141A3183800A25C5B68C9B2FFF7D0FF82
:1018B00000280DD12B78DA00A218013350602B706C
:1018C0003378044A013B3370136A01331362D8E75B
:1018D0000123DFE77066FF1F5C234343074910B510
:1018E000C9180B0058331B78012B05D1FFF7C6FF31
:1018F000034A936A0133936210BDC046A466FF1F7A
:101900007066FF1F10B502F063FB064A0121130049
:1019100010CB4942D967044B136002F081FB2000D1
:1019200010BDC04600E100E01000100010B504003A
:1019300002F04EFB024B1C6002F072FB10BDC04671
:1019400000E100E010B5040002F042FB4021094A2A
:10195000200013688B43136002F0FAFB01F064FD72
:101960000022054B01201A60044B04321A6002F079
:10197000AFFBFEE71CF00040C4F00040C0F00040A8
:10198000431E5A425341A022F0B5D2015B4213409C
:10199000154D164A40019B182A18127E8BB00191F2
:1019A000002A1BD01A000832D46F0022E6B206AF1C
:1019B000E4B294420EDC2818C369002B08D00199C8
:1019C00002AA117106AA049202AA167303A89847E4
:1019D0000BB0F0BD1978B9540132EAE71A7D1A78D4
:1019E00006AB01261A70E6E73069FF1F0040004091
:1019F000F0B5254B04004001C25C85B0002A2BD015
:101A00001A18117E002927D0917E002924D011793F
:101A1000022921D11689D788D168F51BADB22A1CBD
:101A2000102D00D9102292B2BE4217D118180123EE
:101A300003710023C269C38003819A4206D06846BD
:101A4000032103730171029301A890470820002C21
:101A500000D0192001F034FC05B0F0BD013C654216
:101A60006C41A0256442ED012C40084D1B186419FF
:101A7000074D0633013A92B2AA42EDD01888461CAF
:101A80001E80085C2070F5E73069FF1F00400040B1
:101A9000FFFF00000F220E4B10B59868104002386F
:101AA0000A280BD802F0D8F80D0A0B0A0A110A0A04
:101AB0000A0A060002210020FFF762FF10BD012183
:101AC000F9E70020FFF794FFF8E7DB6FF6E7C04681
:101AD000004000400F220E4B10B5986810400238AD
:101AE0000A280BD802F0B8F80E0A0B0A0A120A0AE2
:101AF0000A0A060002210120FFF742FF10BD012162
:101B00000800F9E70120FFF773FFF7E7DB6FF5E760
:101B10000090004013B5334C2378072B3DD8324B4F
:101B20001A78324B002A39D18022196852020A43AE
:101B30001A60252001F034FF20232D4A11680B4341
:101B4000802113606B460422C905086807331042E0
:101B500028D080210422C905C86810422ED08021D7
:101B60002020C905CA688243CA6014221A701A78F4
:101B7000002A2FD18021C905C86820320243CA60DB
:101B800014221A701A78002A28D11A4B1A7D22784A
:101B90005A601D221A705932DA6013BD1A6816494C
:101BA0000A40C5E7086802430A6014221A701A78CE
:101BB000002ACED01A78013AD2B2F7E7C8680243B9
:101BC000CA6014221A7019784A1ED2B21A700029FB
:101BD000F9D1C4E71A78013AD2B2C7E71A78013AC4
:101BE000D2B2CEE7C044FF1F8845FF1F3CF0004043
:101BF000B844FF1F00200040FFFFFEFF564B70B5AA
:101C00001B68012B03D1554A936D0133936502F094
:101C100007F9534B534A1860534B544C1A60012335
:101C2000534A1360534A13602378002B06D00622D0
:101C30005149524802F0A4F800232370504A514BF6
:101C400010681B78C1B2002B0ED14F4CC0B2237864
:101C50005BB2002B4FDB237824785BB264B21B04A9
:101C600024021B191B1813600B1C50294ED950233A
:101C7000464A47491078DBB2FF2202284BD1086858
:101C8000444C454D267890432A78964254D9227880
:101C900024782E78023B5D10A31B6B435201D31AAC
:101CA00010335B111843086002F0D2F9031F012BB7
:101CB00045D83A4B1B78002B06D0394B1B78002BAC
:101CC00002D0002002F06CFAA122364B92009978E3
:101CD000354B4A431B689B18832292009B181B7844
:101CE000033B012B03D8AF20400002F041F8012252
:101CF0002E4BDA8270BD237824785BB264B2FF3356
:101D0000FF341B0424021B190138ABE7CAB2022AB4
:101D1000AED20223ACE70868254C264D26789043C6
:101D20002A78964208D9227824782D78023B5B10D5
:101D3000641B63435201B2E72378DBB2B2E70228A7
:101D4000D5D11D4B1B78013B022B03D91B4B1B78B4
:101D5000022BCCD16C20C8E79809FF1FFC0FFF1F96
:101D6000A865FF1FFF3F000014100340AC65FF1F74
:101D70000C10034000100340D50BFF1F7211FF1F12
:101D8000B40003408C09FF1F680AFF1F490AFF1FA8
:101D900094000340460AFF1F470AFF1FF908FF1F70
:101DA0002209FF1F300DFF1F3409FF1FBC0BFF1F4F
:101DB000440AFF1F450AFF1F1C09FF1F2309FF1FBD
:101DC00010B501F065FF0022014B1A8010BDC0461E
:101DD000A465FF1F10B501F0BBFFA121054A8900D2
:101DE0009478054A61431268044B5218528C1A8049
:101DF00010BDC046300DFF1F3409FF1FA465FF1F33
:101E000010B50D4B0D4A9978A1239B004B431268E6
:101E1000D218531DD97F0A4B1B88994209D2441C02
:101E200007D0C82805D0D2695B1A5A43054B5343E3
:101E3000C01802F035F810BD300DFF1F3409FF1F28
:101E4000A465FF1F7102000070B5244D2B68002BA4
:101E500028D001F04DFF2B68D8402B680400002BE0
:101E600027D002F065F82B68D8401D4B1D4A9978A1
:101E7000A1239B004B431268D118D25C91239B0095
:101E8000002A20D0CA580132CA50174B17491B6884
:101E90000868834214D3D23B181A012A1AD0144B73
:101EA000186070BD01F024FF124B196802F0F8F8B9
:101EB000D3E702F03DF80F4B196802F0F1F8D4E7D0
:101EC0000D495B18E8E7CA500C4B1B68DB68E41847
:101ED000201AE4E7F530FF30E1E7C0461C08FF1F99
:101EE000300DFF1F3409FF1F9C09FF1FA865FF1F4E
:101EF000A009FF1F1808FF1F2DFF3F00B065FF1F3F
:101F000070B504000D00282916D10300A433C2883F
:101F10001B889B1A0B4A9BB293420DD906006A3666
:101F200005223100653001F083FF002804D1310023
:101F3000200001F0C5FE70BD2900200001F028FF3F
:101F4000F9E7C046FE7F0000F8B50400012001F06B
:101F50004FFF02F0ADF8174A1749106009680300F7
:101F60001648174E01601748776805680020AF4291
:101F700001D27068281A144D091928601348C162EB
:101F8000A421446A49032143416211490978002987
:101F900005D010490978022902D10F3B1360F8BD22
:101FA000012901D1083BF9E7032901D1053BF5E7F8
:101FB000033BF3E7E408FF1F28F00040340AFF1F4B
:101FC00028100040180AFF1F1C0AFF1F00F00040E5
:101FD0001C09FF1F4A0AFF1F70B580241025E40565
:101FE000A3682B43A36001F0D3FFA368AB43A360B6
:101FF00070BD0000F7B5160080221C001023D2052A
:102000000191916805000B43936000225A4BD73031
:102010001A6002F055F89D232A002F009B00EB5810
:10202000CA3201210092FC37002B01D00021009A16
:10203000386801F015FF2900009BCB311A784F4B0F
:10204000D3351A604B780A781B0213438A7812043E
:102050001A43CB781B061343494A1BBA13604B79CA
:102060000A791B0213438A7912041A43CB7931008F
:102070001B061343434A1BBA13606B782A781B0272
:102080001343AA7812041A43EB781B0613433E4A03
:102090001BBA1360019A330213433C4A13603C4B52
:1020A00022001B1B9C4603293DDCB3089A00130049
:1020B0005142B21A032A46D1354AE018511A8278A1
:1020C0004078120400020243E05C043302430A60D9
:1020D0000022FF2B4BDDF0222E4B12011A600F2243
:1020E0002D4B1A602D4A1368002BFCD00023224A86
:1020F00027491360091B321D0B191B68043A180A83
:1021000023706070180C1B0EA070E3700434002A5A
:10211000F2DC802210213B68D20501333B609368DA
:102120008B439360F7BD6346D578981893782D0656
:102130001B042B43157804392B43557804322D02A8
:102140002B430360AFE7022A0AD1114AE05C511A1F
:10215000E2185278120202430A6004339BB2B7E7D6
:10216000012AB5D10A4A521AE15C1160F5E7084923
:1021700059180A600433ACE7000004403C000440F6
:102180003800044034000440300004400C00044097
:102190000001044004000440100004401400044006
:1021A000F7B5150080221C001023D205009191681C
:1021B00007000B4393600023654AD730136001F09A
:1021C0007FFF9D233E009B00F9583B00CA3632003A
:1021D000FC33002900D07FE0586801F041FE39004F
:1021E00032785C4BCB311A604B780A781B02134370
:1021F0008A78AC4612041A43CB78281D1B06134379
:10220000554A1BBA13604B790A791B0213438A792A
:1022100012041A43CB791B061343504A1BBA1360AE
:102220004B7A0A7A1B0213438A7A12041A43CB7A36
:1022300021001B0613434A4A1BBA1360009A2B0263
:102240001343484A13602200474B1B1B0093009B1B
:10225000CE785B1801938B7836061B0433430E78D7
:10226000043833434E78043136023343019E3360E1
:102270000328ECDC0321A808431C9B0029408000B4
:1022800003292BD13849E5185E18A9786D78E35CED
:1022900009042D022943194331600300083300214A
:1022A000FF2B2DDD314B324919600F21314B196065
:1022B000012327490B60304B19680029FCD0062107
:1022C0001B680B40042B20D080220020D20593688D
:1022D0000A318B439360FEBD01217DE7022908D1BD
:1022E00021495D18E1184978E35C09021943296026
:1022F000D3E70129D3D11C495918E35C0B60CCE723
:102300001948181801600433CAE7002310490B600C
:102310006346002B0CDC3B00FC335A681021013271
:102320005A608022D205936801208B439360D2E7E4
:10233000009B9B181B68190A13705170190C1B0E17
:10234000D37004235B4291709C440432E0E7C046A2
:10235000000004403C0004403800044034000440C5
:10236000300004400C00044000010440040004401C
:10237000080F0000100004401400044070B5061E51
:1023800019D00222614B9B799343012B13D1604BEF
:102390001A78FF2A0FD15A78FF2A0CD19A78FF2A8F
:1023A00009D1DA78FF2A06D11A79FF2A03D15B799D
:1023B000FF2B00D1A7E0574B0C201A78012A08D038
:1023C0000022554D1A702B781A00093A042A01D8B8
:1023D000212070BD5A1F012AFAD94C4CA07B042839
:1023E00000D990E0A279032A00D98CE0821E012A4C
:1023F00003D862881F2A00D885E0002E61D0012E04
:1024000000D080E0A288012AE2D0002B0AD1013856
:10241000032803D801F020FC151D19151F202E706C
:1024200001F04EFD2B785A1E032A16D800253B4B8F
:102430001D602823237501F0ABFEA8422ED0A58095
:10244000C6E7022320202B70EAE7042322202B700A
:10245000E6E7032321202B70E2E7073B012BB7D8E7
:102460002F4B1B68DB6A9B06B2D52E4B1A78002ACD
:10247000AED1A27B911E012901D9002AA8D1022246
:1024800080211A702823284D89012878237501F0AE
:10249000BFFD80212878890101F03AFD0123A38046
:1024A000224B1B78002B0AD0FA228021204B92006D
:1024B0001B8809025A431C4B187801F079FC002054
:1024C00087E701F085FD2B78A680073B012B06D915
:1024D00018482E7001F084FD1E2001F0F1FC114B14
:1024E000114C1A78002A06D0802100222078890118
:1024F0001A7001F08DFD01F093FD80212078090212
:1025000001F086FDDBE7122063E7C046A60BFF1F44
:102510006B09FF1F1A09FF1F1C09FF1F4809FF1F36
:10252000B065FF1F2309FF1F1B09FF1F2109FF1FA4
:102530002C09FF1F0010004010B5002901D001F048
:102540007FFD10BDF7B5604B01919978A1239B00E9
:102550004B435E4A060014681022E418D6235B0041
:10256000E0583623FF33E35C00279343222B41D10D
:10257000574B0F3A1A600760012501F0D9FB019B08
:102580001880E8235B00E35C002B01D0B34258DDE8
:102590000023504FFB70AD33FF33E3581A68002A15
:1025A00003D09B88DB439B071DD03823FF33E35CBC
:1025B000002B18D09B235B00E35C002B13D1D1339D
:1025C000FF33E35CB3420EDAA4235B00E15AE01868
:1025D000090A023101F08CFC23000122FE33013E86
:1025E00001351A87FA70E8235B00E35C002B2AD0E0
:1025F000A8B2FEBD03683D00002BBED08188043028
:10260000090A023101F074FCD6235B00E3581F6015
:10261000B2E72300B133BA00FF33985801378188FD
:102620000430090A023101F063FCE8235B00E35C3B
:10263000BB42EEDCE822F61AED1800235200A35448
:10264000A6E70027F1E7200001F0E2FB00281FD0F9
:10265000002E1DDD7319882647190193B60020004E
:1026600001F0F6FB5A30800020184068013581885F
:102670000430090A023101F03BFC200001F080FD2A
:10268000A3590133A351BD4202D0019B9D42E6D123
:10269000114BE35C002BABD095239B00E35C002B3C
:1026A000A6D00E4BE15A0029A2D00D4AA35C994254
:1026B00002D90133A3549BE700231A212000A3541D
:1026C00001F05EFC94E7C046300DFF1F3409FF1F88
:1026D00000140340E010FF1F5A02000072020000C5
:1026E0005E020000F8B51D4B1D4F1A78002A10D16C
:1026F000BA7B002A02D101321A7003E0032AFAD011
:10270000022AF8D001F044FD00220120154B1A7076
:10271000F8BD154B154D1C68154B9E7801232B7089
:102720002878C0B200F0DEFCBB7B002B0BD101F09F
:10273000D7FAA1239B007343E41883239B00E4187A
:1027400023782B70E4E7032B02D101F099FCF0E72A
:102750000020022BDCD101F02BFCEAE71C09FF1F53
:10276000A60BFF1F2309FF1F3409FF1F490AFF1F84
:10277000300DFF1FF0B587B00EAD2F780FAD2D785F
:102780000593AC46634614000E4D0CAA12782E78C1
:1027900003930D9B009201932200059B029701F089
:1027A0002FFC2E70012C01D0042C08D18022064968
:1027B0008B889343054A1278D20113438B8007B06C
:1027C000F0BDC0461C09FF1F6C11FF1F7809FF1FD9
:1027D0000B001B3B70B504003020E02B0DD813001C
:1027E000E025493BFF3B9BB2ED00AB4205D8034BD4
:1027F000200019825A8201F0A3FC70BD8410FF1FD3
:1028000010B501F00DFB054B00205B68052B04D9CA
:10281000034A5268D20200D4980810BD001000404C
:10282000FCE100E070B501F0D3FB0D4B1B68FC33FD
:10283000DC691D6AFFF7E4FF6419844204D2094B86
:1028400001241B68002B07D004220024064B1A70B9
:10285000064A93690133936101F0E2FB200070BDE9
:10286000B065FF1F9809FF1F2309FF1FFC0FFF1F03
:1028700070B50C4D2B68FC335C6A01F0A9FBFFF7C7
:10288000BFFF2B680025FC339B6AE318834204D208
:10289000054B1B68AB4200D1051B01F0C1FB2800B2
:1028A00070BDC046B065FF1F9809FF1FD722044BBB
:1028B00092009B5810B5002B00D0984710BDC04621
:1028C0000000FF1FF0B587B001F050F9FFF7EEFFF1
:1028D000CA4BCB4C04931B78022B45D1C94B1B68C8
:1028E000186A01F085FAC84BC84A1A60C84BC94A31
:1028F0001A60A022C84B52001A60049B187801F09D
:102900004FFBC649C64801F0FBFBC649C64801F06B
:10291000F7FB1022C54BFF201A60802252031A6079
:10292000802292031A60802212041A6001F038FC9F
:10293000012001F0F5FAFA20400001F0D1FA582008
:1029400001F016FABA4801F0F3FB012001F040FA59
:10295000072001F005FA2268B64B1A4084235B0079
:102960001343236007B0F0BD01F022FCB24E029089
:10297000322001F03DFA33681B0629D43C2001F0D7
:1029800037FA0F2001F034FA9C4B1B78012B00D151
:102990001EE180223368A94D134200D0A7E02B68C6
:1029A000032013432B6001F023FA01F001FC029B8A
:1029B0000299C31A5A1E814200D81A00A04B1A600D
:1029C000904B19681E2353439E4A9B18CB618AE79C
:1029D00001F0EEFB80239C4ADB02116803900B435D
:1029E00013602268934B994F1A40282313432360A6
:1029F000032001F0FDF903203D6801F0F9F93B687F
:102A00000320DB03DB0B009301F0F2F93B68ED03DD
:102A1000DB03ED0BDB0B8E4A0193AB18C22B30D8D6
:102A2000009B9B18C22B2CD8019B9B18C22B28D82B
:102A3000009B2A009D4200D21A00009B9D4200D9B3
:102A40001D00019B934200D21300019A954200D9C8
:102A500015005B1B122B14D80C22336814209343EF
:102A6000336033687B4A1340336001F0C1F90821B9
:102A70003B682268DB038A432260774ADB0B1360E2
:102A80007FE7032001F0B4F93B68DB03DB0B059320
:102A900001F08EFB039B0399C21A531E814200D89A
:102AA00013006E4A93421BD9FF23356869492D0AEA
:102AB0001D4032686B1C1B060A401B0C134333601D
:102AC0000C23326800209A43083B1343336001F023
:102AD00027FB6348634BA840984206DCFEF732FFB1
:102AE000019B009D0093059B95E75F48F6E7002357
:102AF0005E4F554A3B6080231168DB020B43136035
:102B000080222B68032013432B6001F071F93B688E
:102B1000052601333B6080232A685B0213432B6048
:102B20002268444B03201A40514B1343236001F0A9
:102B30005FF90821454B1A682368D2038B43236051
:102B4000454B023900931B68D20B4B439A420CD879
:102B50009B1A3B2B0BD8236846490B4023602B68FC
:102B60000B402B60444B1A601FE7D31AF1E7013E7C
:102B7000F6B2002ED4D123683E4A134023602B685E
:102B800013402B603B68042B07D9BFF34F8F3B4B9F
:102B90003B4ADA60BFF34F8FFEE780222B680320A9
:102BA00093432B6001F024F92268224B03201A4042
:102BB00028231343236001F01BF9244B009A1B6860
:102BC000DB03DB0B1360082223689343236097E742
:102BD00007222C4D2B681340012B02D1002001F05D
:102BE000DFF9AB68284A02201340AB6001F000F91E
:102BF0008023AA685B001343AB60D6E64A0AFF1F36
:102C00005CF00040B065FF1F000003400180063DFE
:102C1000BC00034034080000A4000340710200001F
:102C200014100040FFFF3F002810004000E100E0CA
:102C30003075000000FEFEFFC4F0004044F000408C
:102C40009865FF1F7206000040F0004064F00040ED
:102C500091FCFFFFFF00FFFFA065FF1FE30C0000DA
:102C6000E88000005F361E0060361E002444FF1F0F
:102C700028000100FFFFFEFF9C65FF1F00ED00E044
:102C80000400FA053CF00040FFFEFFFF694E336888
:102C900088331B6883F3088801F03AFA00F0C4FB1C
:102CA000654B664A1B68934207D0002001F038FA52
:102CB0000221634A13688B431360FFF703FE614BE5
:102CC000614C1878C0B201F053FA0023A3600233BC
:102CD000A3605E4B0120236001F08AF80323A36008
:102CE00001F066FA040001F09BF8050001F060FABB
:102CF000574B186000F0D4FF564B1968621A531EE8
:102D0000A14200D213008022D203934201D39B023E
:102D10009B0A3268D16AC90700D478E04E491C0C7E
:102D200009689BB24C4359432402090A64180327DB
:102D30004A49FC3293680A6849489B1A494A4A4EF4
:102D400012684A499B18414A34609A183B400193E3
:102D5000036892089C46019B0A6063440360042B4D
:102D600003D901323B400A6003600B684049E41814
:102D7000200001F095F93F4F3D493B68C3183B6087
:102D80002000019300F0CCFF3B4C20680818384924
:102D90002060884205D9019B01333B6000F0C0FFF1
:102DA000216000F095FF354B1B78002B0ED001F011
:102DB00037F83168324B4A1B1B6812189A4233D2DB
:102DC000591A4919091A2F4801F09AF92E4C237AF9
:102DD000002B0FD001F024F83168E3684A1B121869
:102DE000934224D9591A4919091A284801F088F937
:102DF00000232372264B83F3088800F0A1FF0220F2
:102E000001F05EF8002001F08BF901F031F9DC01EE
:102E100099000234641A5900641A09214B43803323
:102E2000CB40A408E41882E7FA218900CBE71949CE
:102E3000DBE7C046B065FF1F0C0AFF1FB641210348
:102E400010000040490AFF1F14100040C409000090
:102E5000100AFF1F340AFF1F380AFF1F200AFF1F36
:102E6000280AFF1F1C0AFF1F9465FF1F240AFF1F6B
:102E7000710200006008FF1F2C0AFF1F1C09FF1FC2
:102E8000E408FF1F00100040740BFF1F3C100040BF
:102E900000000020DC050000A022054B92009B589A
:102EA00010B5002B01D0984710BD01F089F8FBE761
:102EB0000000FF1FA122054B92009B5810B5002B6C
:102EC00001D0984710BD01F07BF8FBE70000FF1F21
:102ED000A222054B92009B5810B5002B01D09847B9
:102EE00010BD01F06DF8FBE70000FF1FA322054BAA
:102EF00092009B5810B5002B01D0984710BD01F0EF
:102F00005FF8FBE70000FF1FA422054B92009B58CF
:102F100010B5002B01D0984710BD01F051F8FBE728
:102F20000000FF1F70B500F07BFF514B18600420BC
:102F300000F0C6FF00F0ACFF0400C30702D401F0AC
:102F4000D7F870BD00224B4B1A604B4B18780138F4
:102F500004282CD800F080FE03231B1F270020002C
:102F600001F046F80128ECD0444C2378042B71D1B1
:102F700000F086FF002806D001F0F2F8582000F09B
:102F8000F7FE02232370032000F09AFFD9E7200008
:102F900000F0B6FEE6E7200000F0EAFFE2E72000DE
:102FA00001F09EF8DEE7200000F01AFFDAE701F0FA
:102FB0004FF80500012808D1314B1B78053B012B48
:102FC00003D82000FFF768FFCEE72C4B1B78022BBD
:102FD00001D0052B20D1022D28D12A4B9B7BAB435E
:102FE0001CD12000FFF766FF254B18780128BBD1C4
:102FF0006405B9D4234925224B7B034205D1233AEA
:1030000013405A42534126331A000B7D9342ABD9E9
:10301000322000F0C5FEA7E7022D07D1184B1B7820
:10302000052B11D12000FFF753FFDDE7012D0BD158
:10303000012B03D12000FFF759FF95E7062B03D1A1
:103040002000FFF761FF8FE7200000F0B9FF022D9D
:103050008AD1C9E7032B04D10B4B987C00F008FF01
:1030600091E7072B8FD1094B987B00F0F9FF8AE796
:103070009C09FF1F9809FF1F9009FF1F2309FF1FCD
:103080001C09FF1FA60BFF1FBC0BFF1FD40BFF1F4C
:10309000FA210A4B0A4A49001A640A4A5A500A4A53
:1030A00004395A50094A08319A64094A5A50094A5F
:1030B0005C315A50084ADA667047C0460000FF1F6C
:1030C0007527FF1F7128FF1F2528FF1F7D23FF1F66
:1030D000E526FF1F011EFF1FD51DFF1F10B500F0C5
:1030E000A3FD10BD8023F7B59C46264B264F0193C8
:1030F0002649274A274D284C284B02281AD16046DA
:1031000038600868264E3040802636033043086019
:1031100001990978002909D11660224A2A60224AB9
:103120002260E02219689143A03A1BE08021C90285
:103130001160F2E766463E600F68194E3E408027F8
:10314000FF023E430E600199097800290DD11760F6
:1031500001280ED1154A2A60154A2260E02219681A
:103160009143C03A0A431A60F7BD80218902116079
:10317000EEE7E0210F4A02432A600F4A22601A68F4
:103180008A43F0E74B0AFF1FE0000340D8000340EA
:103190009000034000000340500003404000034003
:1031A000FFFFE3FF0280063D804508220180063DC7
:1031B000806608220080069880550822F8B51E4BCC
:1031C00080261A68002014003440324232D11A6836
:1031D0001A4F32431A6001223B68063093433B602A
:1031E00000F006FE0122164D2B681E432E603B6840
:1031F0000A2613433B608027BF00124B1B683B42EB
:1032000011D1013EF6B2FF2E09D17E220E4B1C6871
:103210002B68E40B1440934323432B6005E0082004
:1032200000F0E6FDE9E7002EEFD180222B68600870
:1032300093432B60F8BDC046C4F000405CF00040F2
:1032400018F0004068F0004060F0004010B500F059
:1032500087FE01215820034A00F0B2FFFFF7AEFFBE
:1032600010BDC046600AFF1F10B578220021034838
:1032700000F006FD00F0DCFE002010BDB868FF1F66
:1032800070B5040000F0A4FE00230C200B4A0100DE
:1032900059438D18515C00290DD0A14208D101235A
:1032A00000246B7000F054FE00F0BAFE200070BDE8
:1032B00001330A2BEBD11224F6E7C046B868FF1F92
:1032C00070B5040000F084FE002319001D000D4AB3
:1032D0001078002806D0A0420CD1557001310C3274
:1032E0000A29F5D1002B0AD100F0A2FE00F098FEC9
:1032F000002070BD5078461EB0411B18EEE700F06C
:1033000027FEF3E7B868FF1FF7B504000C20002381
:1033100084460E4D019267465F43E85D7E19A042E8
:1033200012D000280BD10A4B9C4662461B7808330A
:103330001370019B70707C557160B360FEBD0133EA
:103340000A2BE8D10320F9E70720F7E7B868FF1F49
:10335000B468FF1F8021204BC9051B6870B58B60C6
:103360001E4BC1241A680123FF2013434B611C4BE1
:10337000A4001A681B4B00251A601B4B1A681B4BD4
:103380001A601B4B1A5982431A51C52292009C584D
:103390008443BF38204398509C58164804408020EE
:1033A000C001204398509858134C0002000A014372
:1033B0009950124B1B78DB08AB4201DC002070BD3A
:1033C0002378002B06D0A368002B00D09847013546
:1033D0000C34EEE71220F2E7BC44FF1FB844FF1F95
:1033E000B0F00040B068FF1FB4F00040AC68FF1FB1
:1033F00000E100E0FF00FFFFB868FF1FB468FF1F97
:10340000030010B51F2809D8072200201340072405
:1034100004490A78A24313430B7010BD0023062011
:10342000F5E7C046B468FF1F034A0449136800204B
:103430000B4013607047C0461CF00040FFFFC1FF07
:10344000054B06491B780A6805485B0702401B0BC1
:10345000134300200B607047B468FF1F1CF000404E
:10346000FFFFC1FF70B50C25FFF7EAFF0A4B1C7880
:103470000A4BE4086543ED18002C01D1200070BD13
:103480002B78002B06D06B68002B00D09847013CAE
:103490000C3DF1E71220F2E7B468FF1FAC68FF1F94
:1034A00007B50422074801A900F034F9019B013354
:1034B00005D18023044ADB0411680B43136000200C
:1034C0000EBDC0461C18001114F00040F0B50500F8
:1034D0002026184B87B00493049B002B03D11124A2
:1034E000200007B0F0BD002102220B0001910091E5
:1034F000052000F065FC02230F490A681A42FCD13E
:103500000596059C631E0593002CFAD10B4A13689F
:10351000002BFCDA0F276F440121380000F0B8FDC2
:103520003B782B42DCD0052000F062FC049B013B81
:103530000493D1E7FFFFFF0790C8004000C8004098
:1035400007B500F045FD80220821D205936A01915C
:10355000002B01D10739916202210C4A11600199B7
:10356000481E01900029FAD1033111600531019103
:103570000199481E01900029FAD11160002B02D157
:103580008022D205936200F04BFD07BD00C00040D1
:10359000F0B52D4C89B02378002B4FD1FEF7B2F94E
:1035A00002232A4F03903A681A42FCD12023069343
:1035B000069B5A1E0692002BFAD1254E3368002B2B
:1035C000FCDA0120FFF782FF011E02D0112009B0B2
:1035D000F0BD030003220190009005AD9F2000F094
:1035E000EFFB0321280000F053FD02233A681A4242
:1035F000FCD120230793079B5A1E0792002BFAD178
:103600003368002BFCDA0120FFF760FF0028DDD1D2
:103610000398FEF78BF9AA786B7811041B020B4311
:1036200029780B4363601300113B0A49052B07D827
:1036300001239340A3600B60012323700020C6E7A1
:1036400080231B03F6E7C046A444FF1F90C8004038
:1036500000C800409808FF1F1E4B30B55A68187804
:103660001D4B85B0D31859424B41012100930023D3
:1036700000F01EFC194B1A4A02259A6300221A65B3
:1036800010325A658022C4219D65164B1648D2021D
:10369000DA6789004258154B80241A4080231B04A6
:1036A00013434350642341200393E40500F078F969
:1036B000402000F075F96562039D6B1E0393002D99
:1036C000FAD103236362FFF73BFFA562FFF760FFB8
:1036D00005B030BDB044FF1F95FFFEF700C80040A5
:1036E000050001FF04E100E000E100E0FFFF00FF52
:1036F00010B5064B18705960FFF7AEFF002113207C
:10370000034AFFF701FE002010BDC046B044FF1F72
:103710005936FF1FF0B5040085B003920291FEF701
:10372000F1F8882263035B0B52051A438023DB0503
:103730009D6A8023274F0092BA68002601901B03E0
:103740009A420CD9F82326001B041E401C4206D0C6
:103750008022214B52025E6219680A431A60002DD2
:103760000BD100F035FC02221C4B1A608023DB05D4
:103770005A62013A9A6200F053FC0023039A934282
:1037800020D1002D0AD100F023FC144B03221D6030
:103790008023DB055A629D6200F042FC8023BA68F8
:1037A0001B039A4208D9002E06D000220A4B0C496E
:1037B0005A621A680A401A600198FEF7B7F80020AA
:1037C00005B0F0BD009A0299D2181278CA5401339C
:1037D000D4E7C046A444FF1F00C8004000C000401A
:1037E000FFFFFEFFF0B587B0029103920400FEF7E1
:1037F00089F8019000F0ECFB802302250122234E82
:10380000DB0535605D629A6200F00AFC204F3B6880
:103810002B42FCD120230493049B5A1E0492002BBC
:10382000FAD11C4D2B68002BFCDA0120FFF74EFE6D
:10383000002802D0112007B0F0BD2000039A0299A1
:1038400000F046FB022304003A681A42FCD1202310
:103850000593059B5A1E0592002BFAD12B68002B6D
:10386000FCDA0120FFF732FE051EE3D100F0B0FBC9
:1038700080230322DB0535605A629D6200F0D0FB95
:103880000198FEF753F8E0B2D5E7C04600C000400B
:1038900090C8004000C80040F0B5802687B0040002
:1038A000FEF730F8F605B36A02250393029000F0A4
:1038B0008FFB0123244F3D607562B36200F0B0FBC3
:1038C000224E33682B42FCD120230493049B5A1EC2
:1038D0000492002BFAD11E4D2B68002BFCDA01203C
:1038E000FFF7F4FD002802D0112007B0F0BD200042
:1038F00000F0DEF90223019032681A42FCD1202345
:103900000593059B5A1E0592002BFAD12B68002BBC
:10391000FCDA0320FFF7DAFD041EE5D100F058FBC6
:1039200080230322DB053C605A629C6200F078FB36
:10393000039B002B01D1FFF703FE0298FDF7F6FF72
:103940006B461879D1E7C04600C0004090C80040DF
:1039500000C8004007B5000201910422000A01A935
:10396000FFF740FF0EBD000073B5050005240B4AAC
:10397000A3005B429B1819686B46DE1D300000F007
:10398000C7F9022804D133782B55013CEFD276BD1C
:10399000052CFCD00128FAD10230F8E714090011F7
:1039A0001F2807D8012380228340D20591680B434A
:1039B000936070473F2808D8012380222038834035
:1039C000D20551690B435361F3E75F28F1D8012316
:1039D000802240388340D205116A0B431362E8E726
:1039E0001F2807D8012280218240C9058B68934394
:1039F0008B6070473F2808D8012280212038824000
:103A0000C9054B6993434B61F3E75F28F1D8012265
:103A1000802140388240C9050B6A93430B62E8E776
:103A20001F2810D880230200DB05153A1968012AE7
:103A300006D820229143196019680A431A6070471A
:103A400001228240F6E73F2811D880230200DB05DF
:103A5000353AD968032A06D810229143D960D9682B
:103A60000A43DA60EBE7012220388240F5E75F285D
:103A7000E5D842238022181A413B8340D205516A7F
:103A800099435162516A0B435362D8E710B5040061
:103A9000012813D1A022184992050B685B015B092C
:103AA00013430B60154B164A19681140154A0A4317
:103AB0001A60402219680A431A6010BD0028FCD120
:103AC00001000A2000F0BCF921000B2000F0B8F939
:103AD000C0220A4B920019680A4340211A601A68F2
:103AE0008A431A60B022044912060B685B015B0925
:103AF00013430B60E1E7C04614F000401CF00040A7
:103B00007F00FEFF80FD0100FA2110B58900C0038F
:103B100000F0C6FA00F06CF910BD000072B6074A5A
:103B20001368013313600422054B1A600023054A11
:103B300013608022D2055360FEE7C0467808FF1F5D
:103B4000C0F00040C4F00040044B054A1A60054B29
:103B50001A600022044B1A607047C046140AFF1F07
:103B6000841E0000380AFF1FC4F000400023034AEF
:103B70001360034A1360034A1360704754F0004017
:103B800040F1004044F10040002310B5184C8AB0C9
:103B9000009301932378012B27D06946012000F080
:103BA0002FF9002817D1009B12490293019B06AA06
:103BB0000393114B02A81B680493104B1B680593D9
:103BC00000F0E6F910220E4906A800F031F90028AD
:103BD00004D1FF23237000200AB010BD0123094A3D
:103BE000074902A8237000F0D3F90120F4E7C0468A
:103BF000B465FF1F10290011082900110C290011BC
:103C000020290011B865FF1F13B501246946012062
:103C100000F0F6F8034B00940193FFF7B5FF200086
:103C200016BDC046BB0B000010B5FFF79FFFFFF7A6
:103C3000EBFF002802D0024B984710BDFEE7C046BC
:103C4000E1A2000002B47146490849000956490042
:103C50008E4402BC7047C04602B471464908490010
:103C6000095C49008E4402BC7047C04603B47146EB
:103C7000490840004900095A49008E4403BC704776
:103C800001B40248844601BC604700BFB70E000083
:103C900001B40248844601BC604700BF8D82000029
:103CA00001B40248844601BC604700BFC166010000
:103CB00001B40248844601BC604700BFA96F0100FF
:103CC00001B40248844601BC604700BF85C10000C2
:103CD00001B40248844601BC604700BFD5440100DE
:103CE00001B40248844601BC604700BFE9F6000009
:103CF00001B40248844601BC604700BFE90B0100E3
:103D000001B40248844601BC604700BF0934010089
:103D100001B40248844601BC604700BF1538001159
:103D200001B40248844601BC604700BF090E000090
:103D300001B40248844601BC604700BFCD0C0100BD
:103D400001B40248844601BC604700BF7997000077
:103D500001B40248844601BC604700BFF9ED000091
:103D600001B40248844601BC604700BFF90D010060
:103D700001B40248844601BC604700BF79120100CB
:103D800001B40248844601BC604700BFE94C010011
:103D900001B40248844601BC604700BF51B800002E
:103DA00001B40248844601BC604700BF613701008E
:103DB00001B40248844601BC604700BF8B52010039
:103DC00001B40248844601BC604700BF496D010050
:103DD00001B40248844601BC604700BFE5120100FF
:103DE00001B40248844601BC604700BFF9350100B8
:103DF00001B40248844601BC604700BF018900004D
:103E000001B40248844601BC604700BFE1AC000039
:103E100001B40248844601BC604700BF71B0000095
:103E200001B40248844601BC604700BFC95C010080
:103E300001B40248844601BC604700BFCD4C01007C
:103E400001B40248844601BC604700BF919900114B
:103E500001B40248844601BC604700BFD9B00000ED
:103E600001B40248844601BC604700BF2144000001
:103E700001B40248844601BC604700BF4DF9000010
:103E800001B40248844601BC604700BF01D700006E
:103E900001B40248844601BC604700BFBD0B01006D
:103EA00001B40248844601BC604700BF8937010065
:103EB00001B40248844601BC604700BFC56D0100E3
:103EC00001B40248844601BC604700BF19070100E5
:103ED00001B40248844601BC604700BF95730100ED
:103EE00001B40248844601BC604700BF851201004E
:103EF00001B40248844601BC604700BFC1150100FF
:103F000001B40248844601BC604700BFA1AD001166
:103F100001B40248844601BC604700BF0D52010055
:103F200001B40248844601BC604700BF691101002A
:103F300001B40248844601BC604700BF6D0B01001C
:103F400001B40248844601BC604700BFE927000075
:103F500001B40248844601BC604700BF21A90000AB
:103F600001B40248844601BC604700BFED6801000F
:103F700001B40248844601BC604700BF053401001B
:103F800001B40248844601BC604700BF53B9000039
:103F900001B40248844601BC604700BFDD3F000019
:103FA00001B40248844601BC604700BFEDA5000093
:103FB00001B40248844601BC604700BF19FA000002
:103FC00001B40248844601BC604700BFE917010004
:103FD00001B40248844601BC604700BF75A90000D7
:103FE00001B40248844601BC604700BFC1A500007F
:103FF00001B40248844601BC604700BF013401009F
:1040000001B40248844601BC604700BF9D6A0000BD
:1040100001B40248844601BC604700BFB3520100AE
:1040200001B40248844601BC604700BF9DA900005E
:1040300001B40248844601BC604700BFADAE000039
:1040400001B40248844601BC604700BFE9D40000C7
:1040500001B40248844601BC604700BFDD0C01008A
:1040600001B40248844601BC604700BFC1F70000AC
:1040700001B40248844601BC604700BF855201007C
:1040800001B40248844601BC604700BF75F80000D7
:1040900001B40248844601BC604700BF3D71010085
:1040A00001B40248844601BC604700BF090E00000D
:1040B00001B40248844601BC604700BFBD5C0100FA
:1040C00001B40248844601BC604700BF8944000037
:1040D00001B40248844601BC604700BFA1AF0000A4
:1040E00001B40248844601BC604700BFF5350100B9
:1040F00001B40248844601BC604700BFDD0A0100EC
:1041000001B40248844601BC604700BF2D6C010029
:1041100001B40248844601BC604700BFC9A9000041
:1041200001B40248844601BC604700BF016C010035
:1041300001B40248844601BC604700BF8D110100F4
:1041400001B40248844601BC604700BF116E000004
:1041500001B40248844601BC604700BFF9A60000D4
:1041600001B40248844601BC604700BF6DF6000000
:1041700001B40248844601BC604700BF89140100B5
:1041800001B40248844601BC604700BF5976010073
:1041900001B40248844601BC604700BFA9D80000B2
:1041A00001B40248844601BC604700BFED6B0100CA
:1041B00001B40248844601BC604700BF156B010092
:1041C00001B40248844601BC604700BF016701009A
:1041D00002000000AEB600110100000098B400110A
:1041E00002000000AAB60011010000001042FF1FEB
:1041F00002000000A0B40011010000001063FF1FC6
:1042000002000000A8B60011030000008862FF1F32
:104210001200000002000000AEB600110100000014
:10422000E0B4001102000000AAB600110100000075
:10423000DDB4001102000000EAB400110300000028
:10424000C362FF1F02000000A8B6001103000000B7
:10425000D862FF1F02000000AAB600110100000092
:10426000DCB4001102000000E8B4001103000000FB
:104270009962FF1F02000000A8B6001103000000B1
:10428000BA62FF1F02000000AEB60011010000007C
:1042900020B5001102000000AAB6001101000000C4
:1042A0005943FF1F0200000032B500110100000059
:1042B0001BB5001102000000AAB6001101000000A9
:1042C0005843FF1F0200000030B50011010000003C
:1042D000E062FF1F02000000AAB60011010000000A
:1042E0005743FF1F020000002EB50011010000001F
:1042F0000BB5001102000000AAB600110100000079
:104300005643FF1F020000002CB500110100000001
:1043100006B5001102000000AAB60011010000005D
:104320005543FF1F020000002AB5001101000000E4
:1043300001B5001102000000AAB600110100000042
:104340005443FF1F0200000028B5001101000000C7
:10435000FCB40011020202020202000075470011C3
:10436000714700115CB50011900118001800FFFFA3
:104370000701020304050602010600000000000018
:10438000000000000000000000000000000000002D
:10439000000000000000030002000000AEB60011A3
:1043A00001000000DCB5001102000000AAB60011F7
:1043B000010000000844FF1F02000000E6B50011E4
:1043C000010000000A63FF1F02000000A8B60011F0
:1043D000030000006465FF1F02000000AAB6001180
:1043E000010000000844FF1F02000000E4B50011B6
:1043F000010000000C63FF1F02000000A8B60011BE
:10440000030000005C65FF1F1200000000010000B7
:1044100000000111FFFF0000504859360000000065
:1044200000000000010000006DB500110B00050048
:10443000F7000000B4000028002800283075A00014
:10444000A000A000A00000080008E001F00010009B
:10445000100010001000100010005000500050001C
:1044600010001000D0070000000000000F00010045
:104470000500307507001000010081FF00000000FA
:10448000FF000000896B0011916900112167001184
:10449000FFFF0100FF00000085950011019300114E
:1044A0001992001100000000000000000000080048
:1044B000040000003B0001085902E00188212800A7
:1044C000FF00000002000000AEB600110100000075
:1044D00074B7001102000000AAB60011010000002C
:1044E0004145FF1F02000000A6B6001101000000B8
:1044F0007069FF1F02000000AAB600110100000051
:104500004045FF1F02000000A4B60011010000009A
:104510003E45FF1F02000000AAB600110100000086
:104520003C45FF1F02000000A2B600110100000080
:104530003445FF1F1800180000009001020000031E
:104540000202000002000000AEB6001101000000EF
:1045500088B7001102000000AAB600110100000097
:104560008445FF1F02000000A0B6001100000000FB
:104570000000000002000000A8B6001103000000C7
:064580009069FF1F20FFFF
:040000051FFF184180
:00000001FF
